:020000040800F2
:1000000040DD0020E9010008DB4A0008BD3D000892
:10001000D94A0008DD0A0008D99400080000000051
:100020000000000000000000000000005101000876
:100030006F1200080000000095010008718D000893
:10004000030200080302000803020008030200087C
:10005000030200080302000803020008030200086C
:10006000030200080302000803020008030200085C
:1000700003020008091200081512000821120008E6
:100080002D12000803020008030200080302000802
:10009000030200080302000803020008030200082C
:1000A00003020008FD8D0008030200080302000897
:1000B0000302000803020008098E0008030200087A
:1000C00003020008030200080302000803020008FC
:1000D00003020008BD9300081D9400087D940008E9
:1000E00003020008030200080302000803020008DC
:1000F000158E00080302000803020008030200082E
:1001000003020008030200080302000803020008BB
:1001100003020008030200080302000803020008AB
:100120000302000803020008030200083912000855
:10013000DFF810D000F0FCF900480047F59B0008FC
:10014000AFF3008040DD002080F308887047000096
:10015000224B19680868B0E8F00F80F30988BFF3F4
:100160006F8F4FF0000080F311884EF00D0E704736
:100170000000000006480068006880F3088862B646
:1001800061B6BFF34F8FBFF36F8F00DF00BF00BFBB
:1001900008ED00E0EFF30980BFF36F8F0F4B1A6893
:1001A00020E9F00F106008B54FF0500080F311887F
:1001B000BFF34F8FBFF36F8F0BF022F84FF00000AB
:1001C00080F31188BDE8084019680868B0E8F00FAE
:1001D00080F30988BFF36F8F704700BF440A002087
:1001E000EFF3058070470000064880470648004747
:1001F000FEE7FEE7FEE7FEE7FEE7FEE7FEE7FEE7D7
:10020000FEE7FEE7FB8D000831010008202A04DB31
:10021000203A21FA02F00021704721FA02F3D0407F
:10022000C2F120029140084319467047A0F16101D4
:10023000192900D82038704740EA01039B0703D0F2
:1002400009E008C9121F08C0042AFAD203E011F815
:10025000013B00F8013B521EF9D27047D2B201E0D7
:1002600000F8012B491EFBD270470022F6E710B5BB
:1002700013460A4604461946FFF7F0FF204610BD14
:10028000421C10F8011B0029FBD1801A7047F0B402
:1002900080EA0102D40F4200B2EB410F02D20246C3
:1002A000084611464A0042D0C30DDDB2C1F3C75221
:1002B000AD1A202D35DAC1F3160141F4000204B164
:1002C0005242C5F1200602FA06F12A411044B3EB6E
:1002D000D05F23D0C4B1012DA0EBC35009DCF0BC2A
:1002E0004FF0004202EAC352DBB200F5000000F01A
:1002F000F0B8400000F1807000EBC350A0F18070B6
:1003000040EAD170490009E0490841EAC071A0EB18
:10031000C35000F50000400800EBC350F0BC00F0F3
:10032000CFB86142012202EB4101001BF6E7F0BCAD
:10033000704781F00041AAE780F00040A7E780EA1B
:10034000010210B502F00043400022D04A001FD045
:10035000010E01EB1261C0F35600C2F3560240F4E5
:10036000000042F40002A0FB022000047F391404C4
:1003700000D0401C50EA124001D44000491EC2B2D5
:100380000C0604EBD010401C4008802A02D003E089
:10039000002010BD20F00100002900DA00201843E1
:1003A00010BD30B480EA010202F0004530F0004296
:1003B00021F0004013D090B1C30DD40DC2F316014B
:1003C000C0F31600E41A41F4000140F400027D3449
:1003D000914201D3641C00E04900002C02DA30BCD9
:1003E000002070474FF400000023914201D3891A86
:1003F000034340084FEA4101F7D151B1914202D184
:100400004FF0004105E002D24FF0010101E06FF032
:10041000010103EBC450284430BC00F051B8C10FB7
:1004200080EAE0700844CA079623002100F051B822
:1004300096230022114600F04CB800F0004220F054
:100440000040C10DC0F3160040F400007F2901DA1E
:1004500000207047962903DCC1F19601C84001E0F5
:1004600096398840002AF4D04042704720F000407E
:10047000C10DC0F3160040F400007F2901DA00200E
:100480007047962903DCC1F19601C8407047963940
:100490008840704730B50B460146002020220124D9
:1004A00009E021FA02F59D4205D303FA02F5491B42
:1004B00004FA02F52844151EA2F10102F1DC30BD58
:1004C0000029A8BF7047401C490008BF20F0010068
:1004D000704710B4B0FA80FC00FA0CF050EA010446
:1004E00004BF10BC704749B1CCF1200421FA04F4D8
:1004F00011FA0CF118BF012121430843A3EB0C01B1
:10050000CB1D4FEA00614FEA102042BF002010BC13
:10051000704700EBC35010440029A4BF10BC7047C3
:10052000401C490008BF20F0010010BC70470000CB
:10053000064C074D06E0E06840F0010394E8070030
:1005400098471034AC42F6D3FFF7F6FDF8CD00081B
:1005500018CE000870B58D1810F8014B14F0030286
:1005600001D110F8012B231106D110F8013B03E053
:1005700010F8016B01F8016B521EF9D1ABB110F804
:10058000012B04F00C048A1A0C2C03D0A2EB841269
:100590009B1C08E010F8014BA2EB0422F8E712F8CC
:1005A000014B01F8014B5B1EF9D5A942D4D30020C1
:1005B00070BD000010B50B4A51B102B2094C4B1E80
:1005C00001EBC10004EBC0000F2B03D8C28010BDAB
:1005D000508010BD41390E29FBD8A0F58050A0F8FD
:1005E000842210BDC82D0020F0B54FF6FF74A04244
:1005F00001D0A14201D12046F0BD44F250677C00F9
:10060000B84200DB201A40F6E445A84200DD284647
:10061000DFF8C4C04FF4FA76BCF80250A0EB050E28
:10062000B64502DD05F5FA7005E0A5EB000EB6450E
:1006300001DDA5F5FA70ACF80200B94200DB611AE1
:10064000012A13DD254F37F81350A1EB050CB445F3
:1006500002DD05F5FA7105E0A5EB010CB44501DDFD
:10066000A5F5FA7127F81310921E1FE01B4F203FCB
:1006700037F81350A1EB050CB44502DD05F5FA710E
:1006800005E0A5EB010CB44501DDA5F5FA71134DAC
:1006900027F81310203503EBC30305EBC303814296
:1006A00002DB091AD98001E0401AD8806AB10844F7
:1006B000A04202DBA0F50C40A03846F67811884233
:1006C0009ADDA0F50C40A038F0BD081A44F2506144
:1006D000C842F2DA2044F0E720030020A82D0020D1
:1006E0002DE9F047284E00258A4604463F2802DDC2
:1006F000A4F1400509E0012C07D01E2C02DBA4F177
:10070000300502E004EBD470451005EBC5008046CF
:1007100006EBC00936F8380009EBC0071B48F86043
:1007200047F8080F7088A0F57F41FF391FD0B6F950
:100730000410491C08D00AF04002B9F904102B46F5
:10074000921CFFF751FF386004EBC40006EBC000B9
:10075000A0F58050B0F98602401C08D00AF02002B3
:10076000B9F9061070882B46FFF73EFF786036F81F
:100770003800401C81B226F83810082902D3002125
:1007800026F83810BDE8F087C82D0020786FFFFFED
:10079000F0B5254D012105F50E63A3F58C6400220B
:1007A000224F3CE0C1EBC10000EB800004EB4000B5
:1007B000C28642869E89012E24D11E8916B1012E41
:1007C0001FD01FE001EBC10605EBC60649F2880EFB
:1007D000D6F814C01CEB0E0F05DCB0F838C00CF1D5
:1007E000010CA0F838C0D6F814E0B4F84260CEF19D
:1007F000000CB44501DCB64503DD068E761C06868A
:1008000000E000BFB0F83CC0B0F84060B44502D38F
:100810000126C68702E0002E00D8C286491C38781F
:100820008142BFDDF0BD0000C82D00202003002064
:10083000F0B58BB005461C4E1C4C28216846FFF7CE
:1008400014FDB4F81D001A4F40BAADF80000207D29
:10085000062804D101223946684600F0BDFD012278
:100860003946684600F0AAFDBDF80000000A287469
:10087000BDF800006874BDF80000A0F57F41FF39A5
:1008800001D0A6F86C00287C617F884206D1687C84
:10089000A17F884202D1207D062802D000200BB023
:1008A000F0BD0120FBE70000A8360020A43700209F
:1008B00050F007082C4B10B52C495A880AB101207A
:1008C00010BD1C7D0022062C12D0B1F87A30FBB18D
:1008D00047217F238174C374FF2404754275817599
:1008E000C375047642768176C3760477427739E021
:1008F0001D480121598046389B7F037006234370B1
:100900008270C1700271082141711948038029E089
:10091000B1F90020120E8274B1F90020120CC274D9
:100920000A88120A02750A784275B1F92820120E57
:100930008275B1F92820120CC2750A8D120A02764E
:1009400091F828204276B1F95020120E8276B1F942
:100950005020120CC276B1F85020120A027791F89A
:1009600050104177002010BDA43700202041002006
:10097000C40900202DE9F0479AB00646A1F1100401
:10098000684603F01DFB00254FF400784FF48069A2
:10099000DFF864A016E000BF05F50070844201D9BD
:1009A000474600E0671B71193A461448FFF744FCBC
:1009B0003A461249684603F085FE3D444946504692
:1009C00002F0B7F8A542E7D3694616A803F0D0FABB
:1009D000002116AA3019535C445CA34203D1491C80
:1009E0001029F8D301E0102903D301201AB0BDE883
:1009F000F0870020FAE70000001001404258002074
:100A0000F0B58BB01F4C28216846FFF72EFC00255F
:100A100001221D49684600F0D1FCBDF800004FF6E8
:100A2000FF760127B04201D0608000E06780082295
:100A30001649684600F0C2FC68460EE030F8151012
:100A4000B14204D004EB4502A2F8441003E004EBE9
:100A50004501A1F844706D1CEDB22188A942EDD882
:100A600000200B4909E000BF04EB40020B88B2F8FC
:100A70004420401C1A440A80C0B222888242F3D823
:100A80000BB0F0BDA836002024F0070860E007088E
:100A9000C60900200F4810B5017D062901D00020AD
:100AA00010BD01210C4C4180817F217006216170B5
:100AB0001221A170C17FE17090F820002071617156
:100AC000A0710821204603F07BF9010AE171207230
:100AD000012010BDA4370020F8370020FEE70000F9
:100AE000F0B58BB00546174C28216846FFF7BDFBD3
:100AF00000216E4605E06018407F26F81100491C71
:100B0000C9B2207E8842F6D8207D0F4F062806D134
:100B1000EA7A3946304600F05FFC00F0BBF8EA7A2A
:100B20003946684600F04AFC002005E016F810102F
:100B30002A18401C1174C0B2217E8142F6D80BB035
:100B40000120F0BDA437002000F007082DE9F05F78
:100B5000484D494C90468B464FF03F46012B06D0FE
:100B6000022B0AD0032B0ED0042B1DD112E0E96C0E
:100B7000FFF7DFFB2062E86213E0696FFFF7D9FB44
:100B8000206268650DE0D5F89C10FFF7D2FB20626B
:100B9000E86706E0D5F8C410A435FFF7CAFB206269
:100BA0002860B04200D926623449206AFFF7C7FBAB
:100BB000FFF75CFC85B2A58000202080D4E905A960
:100BC0002669E069278838F81720AA421CD208EB6A
:100BD00047014A88AA4217D3B9B23BF81100FFF780
:100BE00027FC06460BEB47004088FFF721FC8246B6
:100BF00038F81700FFF71CFC814608EB47004088D7
:100C0000FFF716FC00BF04E07F1CB9B22180C829A1
:100C1000D8D9C4E9046AC4E90690B04652464F46A2
:100C2000064605B341461046FFF783FB8146394629
:100C30003046FFF77EFB06462846FFF7F9FB3946AC
:100C4000FFF777FB3146FFF7ACFB4946FFF777FB31
:100C50004146FFF71CFBFFF709FC6080BDE8F05F31
:100C600080B2FFF7E5BB002020616061A061E06118
:100C7000A080F2E7A03E00205003002000007A444C
:100C800070477047704770477047704770477047AC
:100C9000704770472DE9F04FA1B0E7482090E34C32
:100CA000DFF88C83E34FDFF894B3E54EDFF894A3CD
:100CB00080216846FFF7D9FA00250622E2496846F6
:100CC00000F07CFBBDF800004FF6FF79484514D1D9
:100CD000C822DE49DE4800F07FFBC822DD49DE483D
:100CE00000F07AFBC822DD49DD4800F075FBC82220
:100CF000DC49DD4800F070FB03202080BDF80200D5
:100D000049464FF00109884216D1484606E000BF27
:100D100004EB45026D1C9086A081ADB22288AA42E8
:100D2000F6D80CE004EB4502BDF802009086BDF851
:100D300002006D1CA081ADB22088A842F2D8BDF897
:100D40000400884200D100206081BDF806004A46B8
:100D500088424FF0000006D011E004EB40032282ED
:100D6000401C9A8280B223888342F6D80AE004EBC2
:100D700040052282BDF80630401CAB8280B2238839
:100D80008342F4D8BDF808200D46AA424FF0000077
:100D9000494606D011E004EB40026182401C918478
:100DA00080B222888242F6D80AE004EB40036182D6
:100DB000BDF80820401C9A8480B222888242F4D870
:100DC000A14901222031684600F0F8FABDF8000080
:100DD000A84202D1A4F8089000E020819A4901229B
:100DE0002831684600F0EAFABDF80000A84200D1B8
:100DF00000209549A08001223031684600F0DEFADB
:100E0000BDF80000A0F57F41FF390FD0E080082237
:100E10009649684600F0D2FA00206D4604EB400285
:100E200035F81010082904D2918604E0A4F8069041
:100E3000EDE7A2F83490401C80B20828EED38B492D
:100E400008222039284600F0B9FA002004EB4002BD
:100E500035F81010082901D2918201E0A2F814900F
:100E6000401C80B20828F1D380490822203168460E
:100E700000F0A4FA5FF0000004EB400235F8101017
:100E8000082901D2918401E0A2F82490401C80B28C
:100E90000828F1D36C4901223831684600F08EFAF7
:100EA000BDF80000A0F57F41FF3900D10020664960
:100EB000A4F86E0001224031684600F07FFABDF8C8
:100EC0000000A0F57F41FF3900D10220A4F86400A2
:100ED00008226749684600F071FABDF80010A1F5D4
:100EE0007F40FF384FF0000001D0624A21E000212E
:100EF00007E000BF00EB800206EBC202401C80B29C
:100F0000D16422888242F5D816E000BF35F820105F
:100F10000B0AD370917005EB800149880B0A53705E
:100F200000EB8003117006EBC3031168401C80B214
:100F3000D96421888142E9D8434901224831684671
:100F400000F03CFABDF800004FF6FF75A84202D150
:100F5000A4F8669001E0A4F866003B4901225031F4
:100F6000684600F02BFABDF80000A84202D1A4F8B0
:100F70006C9001E0A4F86C003349012264316846AA
:100F800000F01CFABDF80000A8424FF000001CD190
:100F90005FF00501C0EBC00202EB820308EB4302E5
:100FA000A2F8401000EB001202EB420207EB4202F3
:100FB000401C80B2A2F860100828EBD32098A0F85B
:100FC0004E10ABF87C1031842AE0C0EBC00101EB7D
:100FD000810308EB4301BDF80020A1F8402000EB9D
:100FE000001202EB420207EB4202401CBDF8001067
:100FF00080B2A2F860100828E7D3BDF80000A7F877
:1010000060002098BDF80010A0F84E1000BFBDF899
:101010000010ABF87C10BDF800003084BDF8001063
:10102000AAF87C1021B0BDE8F08F0000A83600209F
:10103000483200203E380020A449002020410020F2
:10104000A03E0020A441002000F0070800D00708BF
:101050008403002000D407081405002000D80708E6
:10106000A406002000DC07083408002020E0070860
:1010700000C007081C0100202DE9F05F5B4EDFF87F
:101080007091DFF870A15C4D4FF0000BF18858466D
:10109000C1B3012934D1594C8903204601F044FDE4
:1010A000A5F852004FF40041204601F03DFD544C9C
:1010B000A5F8A4004021204601F036FDA5F8F60071
:1010C0008021204601F030FDA5F84801A6153146E3
:1010D000204601F029FDA5F89A016115204601F08E
:1010E00023FD484CA5F8EC013146204601F01CFDDB
:1010F000A5F83E02E114204601F016FDA5F8900285
:10110000BDE8F09FFFE7B1880024022922D14FF00B
:101110000008318809E000BF06EB4002401C137D47
:10112000C0B203EB080202F0FF088142F4D80027A6
:101130000EE02046641CE4B200F04AFF07EB071102
:1011400001EB410209EB42017F1CA1F8BE00FFB296
:101150004745EED33089022823D1002080463188CC
:101160000AE000BF06EB4002401C92F83430C0B2E7
:1011700003EB080202F0FF088142F3D800270EE0DB
:101180002046641CE4B200F023FFC7EBC70101EB6B
:1011900081020AEB42017F1CA1F87A00FFB24745A9
:1011A000EED300200746318808E000BF06EB40027E
:1011B000401C92F82420C0B23A44D7B28142F5D8FC
:1011C000002610E02046641CE4B200F001FF06EBAC
:1011D000C60101EB461105EB410202EB4B01761C07
:1011E000A1F85200F6B2BE42ECD389E7A83600203F
:1011F0003E38002048320020A4490020000C014065
:101200000010014000080140014801F033B900001E
:10121000FC2C0020014801F02DB90000742C0020A6
:10122000014801F027B90000302C0020014801F0EE
:1012300021B90000B82C0020014801F01BB90000C2
:10124000EC2B002030B590F840500124AC40C56B29
:101250006C60046863604368102B036803D0996076
:101260000068C26030BD9A600068C16030BD7047E0
:1012700070B500231C4611E011F82350055531F8D4
:1012800023502E0A05196E7051F82360360CAE708B
:1012900051F823605B1C360EEE70241D9442EBD394
:1012A00070BD72B6FEE7000006490020C86106481E
:1012B000016941F004010161016941F040010161EE
:1012C000704700004870002000200240064A0021BC
:1012D000D16106490A6942F002020A61486108695F
:1012E00040F0400008617047487000200020024034
:1012F000044B0022DA61044A136943F001031361CD
:1013000001807047487000200020024014480022ED
:10131000C168CB06134904D5CA6942F00202CA610A
:101320001022C3685B0705D5CB6943F00103CB618D
:1013300042F00402C369DB0707D0CB6943F0040322
:10134000CB61C16921F00101C161A2F58071013950
:1013500001D0C2607047C16921F00101C1617047CD
:10136000002002404870002070B5054601F0EEFBF9
:101370000646114C09E0681C07D025B101F0E6FBD8
:10138000801BA84201D9032070BDE068C007F2D1DC
:10139000E068800601D52020E060E068C00605D442
:1013A000E069C00702D1E068400703D5FFF7AEFF50
:1013B000012070BD002070BD0020024010B507E084
:1013C00011F8014B11F8013B44EA032320F8023BDA
:1013D000521E92B2F4D210BD2DE9F04786B000241F
:1013E000C1F30A06174682468D1B0494009400BF81
:1013F0000120CDE902504FF480694A46294616483B
:10140000FFF7DCFFDFF8508007E000BF3AF8141068
:1014100004EB5602641C28F81210BC42F6D301F00B
:1014200073FA00BF04A9684601F0D0F900BF002498
:101430004F46464605EB440136F8142000230120B0
:1014400001F022FA641CA4B2BC42F3D301F012FAF8
:1014500006B0BDE8F0870000001000202DE9F04F35
:1014600095B004460025DFF834942E4628216846BE
:10147000FEF7FBFE28210AA8FEF7F7FE6F460AA931
:1014800009EB4500884630F8212F52BA27F815207D
:10149000008840BA21F815006D1CEDB2142DEFD371
:1014A00099F81400062816D1FD4D4FF6FF71DFF8AC
:1014B000F4A3287C4FF0000901EA0020697C4FF07A
:1014C000010B0143A87C012906D002297BD0032906
:1014D0007AD0042979D0D8E3012812D002283BD051
:1014E000032854D0042878D0052870D006286FD05F
:1014F00007286ED008286DD009286CD00A286BD038
:10150000C3E31422E8493846FFF766FF1422E64990
:101510006846FFF753FF00204FEA080137F8103004
:1015200031F810209A4201D1761CF6B2401C80B2EC
:101530001428F3D312E20220207525E184F814B0B8
:1015400022E1287C2074687C6074A87CA074E87C0C
:10155000E07484F8149098E3D34914222831384673
:10156000FFF73AFFD049142228316846FFF726FFDB
:101570000020414637F8103031F810209A4201D14E
:10158000761CF6B2401C80B21428F3D3BAE3C649E5
:10159000142250313846FFF71FFFC349142250313F
:1015A0006846FFF70BFF00204FEA080137F81030BC
:1015B00031F810209A4201D1761CF6B2401C80B25C
:1015C0001428F3D3CAE1E3E01DE24AE305E020E09A
:1015D0003BE056E071E08AE0A5E0B349142278319F
:1015E0003846FFF7F9FEB049142278316846FFF714
:1015F000E5FE00204FEA080137F8103031F81020DE
:101600009A4201D1761CF6B2401C80B21428F3D362
:10161000A4E1A5491422A0313846FFF7DDFEA24916
:101620001422A0316846FFF7C9FE00204FEA0801E6
:1016300037F8103031F810209A4201D1761CF6B2FA
:10164000401C80B21428F3D388E197491422C83192
:101650003846FFF7C1FE94491422C8316846FFF7A7
:10166000ADFE00204FEA080137F8103031F81020A5
:101670009A4201D1761CF6B2401C80B21428F3D3F2
:101680006CE189491422F0313846FFF7A5FE8649FE
:101690001422F0316846FFF791FE00204FEA08015E
:1016A00037F8103031F810209A4201D1761CF6B28A
:1016B000401C80B21428F3D350E114227B493846F1
:1016C000FFF78AFE142279496846FFF777FE00206B
:1016D0004FEA080137F8103031F810209A4201D152
:1016E000761CF6B2401C80B21428F3D3E6E36F49AF
:1016F000142228313846FFF76FFE6C491422283136
:101700006846FFF75BFE00204FEA080137F810300B
:1017100031F810209A4201D1761CF6B2401C80B2FA
:101720001428F3D3CAE36149142250313846FFF735
:1017300053FE5E49142250316846FFF73FFE0020F9
:101740004FEA080137F8103031F810209A4201D1E1
:10175000761CF6B2401C80B21428F3D3DEE300BF3F
:10176000BAF80610491C89B2AAF806102A7C22741D
:101770006A7C6274AA7CA274EA7CE2740A296ED044
:1017800084F814B0AAF80690012015B0BDE8F08FD7
:10179000012812D002282AD0032844D004285FD080
:1017A000052877D0062876D0072875D0082874D069
:1017B00009287FD00A287ED067E214223C493846A7
:1017C000FFF70AFE14223A496846FFF7F7FD0020AA
:1017D0004FEA080137F8103031F810209A4201D151
:1017E000761CF6B2401C80B21428F3D366E330496D
:1017F000142228313846FFF7EFFD2D4914222831F5
:101800006846FFF7DBFD00204FEA080137F810308B
:1018100031F810209A4201D1761CF6B2401C80B2F9
:101820001428F3D36EE22249142250313846FFF7D0
:10183000D3FD1F49142250316846FFF7BFFD002039
:101840004FEA080137F8103031F810209A4201D1E0
:10185000761CF6B2401C80B21428F3D32EE362E368
:101860001349142278313846FFF7B6FD1049142287
:1018700078316846FFF7A2FD0020414637F8103066
:1018800031F810209A4201D1761CF6B2401C80B289
:10189000142811E012E02AE045E060E0A4370020BF
:1018A000002400205003002000D0070818D10708AA
:1018B00000D407086FE08AE0E0D3FFE21422FE497B
:1018C0003846FFF789FD1422FB496846FFF776FD8D
:1018D0000020414637F8103031F810209A4201D1EB
:1018E000761CF6B2401C80B21428F3D3E6E2F2492B
:1018F000142228313846FFF76FFDEF4914222831B2
:101900006846FFF75BFD00204FEA080137F810300A
:1019100031F810209A4201D1761CF6B2401C80B2F8
:101920001428F3D3CAE2E449142250313846FFF7B1
:1019300053FDE149142250316846FFF73FFD002076
:101940004FEA080137F8103031F810209A4201D1DF
:10195000761CF6B2401C80B21428F3D3AEE2D6490E
:10196000142278313846FFF737FDD34914227831F5
:101970006846FFF723FD00204FEA080137F81030D2
:1019800031F810209A4201D1761CF6B2401C80B288
:101990001428F3D392E2C8491422A0313846FFF745
:1019A0001BFDC5491422A0316846FFF707FD002042
:1019B0004FEA080137F8103031F810209A4201D16F
:1019C000761CF6B2401C80B21428F3D376E2BA49F2
:1019D0001422C8313846FFF7FFFCB7491422C8313A
:1019E0006846FFF7EBFC00204FEA080137F810309B
:1019F00031F810209A4201D1761CF6B2401C80B218
:101A00001428F3D38AE2012812D0022829D003280F
:101A100043D004285DD005287DD0062876D007283D
:101A200075D0082874D0092873D00A2872D02CE108
:101A30001422A2493846FFF7CFFC14229F4968467A
:101A4000FFF7BCFC0020414637F8103031F8102079
:101A50009A4201D1761CF6B2401C80B21428F3D30E
:101A60002CE29649142228313846FFF7B5FC9349F9
:101A7000142228316846FFF7A1FC00204FEA080134
:101A800037F8103031F810209A4201D1761CF6B2A6
:101A9000401C80B21428F3D334E188491422503119
:101AA0003846FFF799FC8549142250316846FFF704
:101AB00085FC00204FEA080137F8103031F810207B
:101AC0009A4201D1761CF6B2401C80B21428F3D39E
:101AD000F4E17A49142278313846FFF77DFC7749E2
:101AE000142278316846FFF769FC00204FEA0801AC
:101AF00037F8103031F810209A4201D1761CF6B236
:101B0000401C80B21428F3D3D8E104E01FE03AE08F
:101B100055E06EE089E069491422A0313846FFF7AC
:101B20005BFC66491422A0316846FFF747FC0020A1
:101B30004FEA080137F8103031F810209A4201D1ED
:101B4000761CF6B2401C80B21428F3D3B6E15B4990
:101B50001422C8313846FFF73FFC58491422C831D7
:101B60006846FFF72BFC00204FEA080137F81030D9
:101B700031F810209A4201D1761CF6B2401C80B296
:101B80001428F3D39AE14D491422F0313846FFF777
:101B900023FC4A491422F0316846FFF70FFC00206D
:101BA0004FEA080137F8103031F810209A4201D17D
:101BB000761CF6B2401C80B21428F3D37EE11422C6
:101BC0003F493846FFF708FC14223D496846FFF7B5
:101BD000F5FB00204FEA080137F8103031F81020EB
:101BE0009A4201D1761CF6B2401C80B21428F3D37D
:101BF00064E13349142228313846FFF7EDFB3049C0
:101C0000142228316846FFF7D9FB00204FEA08016B
:101C100037F8103031F810209A4201D1761CF6B214
:101C2000401C80B21428F3D348E1254914225031D6
:101C30003846FFF7D1FB2249142250316846FFF79E
:101C4000BDFB00204FEA080137F8103031F81020B2
:101C50009A4201D1761CF6B2401C80B21428F3D30C
:101C60005CE1012813D0022834D003285FD0042877
:101C700079D0052878D0062877D0072876D008288C
:101C800075D0092874D00A2873D000207DE514226D
:101C90000C493846FFF7A0FB14220A496846FFF7B3
:101CA0008DFB00204FEA080137F8103031F8102082
:101CB0009A420AD1761C07E0A0D4070800D807088A
:101CC00018D9070800DC0708F6B2401C80B21428B7
:101CD000EAD3F3E0142295493846FFF77DFB14223E
:101CE00092496846FFF76AFB0020414637F81030FA
:101CF00031F810209A4201D1761CF6B2401C80B215
:101D00001428F3D3142E7FF41CACBAF80610491C27
:101D100089B2AAF80610287C2074687C6074A87CBC
:101D2000A074E87CE07428297FF408AC03E47F49C0
:101D3000142228313846FFF74FFB7C491422283102
:101D40006846FFF73BFB00204FEA080137F81030E8
:101D500031F810209A4201D1761CF6B2401C80B2B4
:101D60001428F3D3AAE005E01FE03AE055E070E064
:101D70008BE0B8E06D49142250313846FFF72CFB58
:101D80006A49142250316846FFF718FB002041468B
:101D900037F8103031F810209A4201D1761CF6B293
:101DA000401C80B21428F3D388E0604914227831B3
:101DB0003846FFF711FB5D49142278316846FFF77A
:101DC000FDFA00204FEA080137F8103031F81020F2
:101DD0009A4201D1761CF6B2401C80B21428F3D38B
:101DE0006CE052491422A0313846FFF7F5FA4F490A
:101DF0001422A0316846FFF7E1FA00204FEA0801FB
:101E000037F8103031F810209A4201D1761CF6B222
:101E1000401C80B21428F3D350E044491422C83146
:101E20003846FFF7D9FA41491422C8316846FFF70E
:101E3000C5FA00204FEA080137F8103031F81020B9
:101E40009A4201D1761CF6B2401C80B21428F3D31A
:101E500034E036491422F0313846FFF7BDFA3349F1
:101E60001422F0316846FFF7A9FA00204FEA080172
:101E700037F8103031F810209A4201D1761CF6B2B2
:101E8000401C80B21428F3D318E0142228493846A5
:101E9000FFF7A2FA142226496846FFF78FFA0020BE
:101EA0004FEA080137F8103031F810209A4201D17A
:101EB000761CF6B2401C80B21428F3D3142E7FF4A3
:101EC00040ABBAF80610491C89B2AAF80610287C63
:101ED0002074687C6074A87CA074E87CE0740A2993
:101EE0007FF42CAB22E71249142228313846FFF741
:101EF00073FA0F49142228316846FFF75FFA002071
:101F00004FEA080137F8103031F810209A4201D119
:101F1000761CF6B2401C80B21428F3D3142E3FF482
:101F20001FACFFF70EBB022121752BE428DC07084C
:101F300040DD070870B51E4C1C4D6078032801D0A9
:101F400006280DD1A078022803D10521184801F0F8
:101F500037FF6078032804D0062801D1E078E070CC
:101F600070BD2078012100EB800202EB801005EBB0
:101F70004000A0F5A040A0F8881B2078E17800EB95
:101F8000800202EB801005EB4000A0F5A040A0F815
:101F9000001B2078217900EB800202EB801005EB1A
:101FA0004000A0F5A040A0F8281B70BDC44E002042
:101FB00000280020054900EBC00202EB401031F878
:101FC000100008B10020704701207047A44900208C
:101FD000F0B4134B114C9915124D08281BD2DFE8B1
:101FE00000F004070B0D0E1013174FF4804101E0B1
:101FF0004FF40041204608E0402100E080211846CF
:1020000003E04FF40071FAE72846F0BC00F08CBD05
:102010004FF40061F8E7F0BC70470000000C01408D
:1020200000100140000801402DE9F0411E4C1D4DFB
:102030001E4F6079A179012641EA002860780328C3
:1020400001D0062808D1A078022805D1052116481C
:1020500001F0B6FE404500D03E80207800EB001134
:10206000C1EBC01005EB4000A0F5E040A0F8B66160
:102070002078E17800EB0012C2EBC01005EB4000C5
:10208000A0F5E040A0F814112078217900EB0012AF
:10209000C2EBC01005EB4000A0F5E040A0F83C11F9
:1020A000BDE8F0816457002000280020C809002006
:1020B00030B53B48394901230078002400EBC002C9
:1020C00002EB401001EB4000A0F58050A0F8103664
:1020D00034480278212A09D0222A07D0232A01D0A5
:1020E000242A0AD14578032D03D129E04578032D10
:1020F00004D0062D01D1C178C17030BD02EBC205FC
:1021000005EB421201EB4202A2F58052A2F80A4608
:10211000027802EBC20404EB421201EB4202A2F588
:102120008052A2F81036C278007800EBC00303EBAF
:10213000401001EB4000A0F58050A0F8C0252AE037
:1021400002EBC20505EB421201EB4202A2F58052FE
:10215000A2F80A46027802EBC20404EB421201EB39
:102160004202A2F58052A2F81036027802EBC204B5
:1021700004EB421201EB4202A2F58052A2F83E3576
:10218000007800EBC00202EB401001EB4000A0F52C
:102190008050A0F85E3500BF30BD0000A44900208B
:1021A000FC0E00200028002010B5040002D0607949
:1021B00010B106E0012010BD00202071204600F083
:1021C00005F801206071002010BD000008B500680E
:1021D0000649884208D10648416941F04001416101
:1021E000406900F04000009008BD0000003002404F
:1021F0000010024070B54379012B20D001254571B4
:10220000022303710668346802F0100340F6FE7280
:102210009A409443D1E900210A439A402243326014
:1022200002681468C02199408C43146002681368E6
:102230008B431360057100214171084670BD022077
:1022400070BD70B5040003D02079002510B105E001
:10225000012070BD6571204600F008F80220207151
:10226000256101202071002070BD0000F0B585B00F
:1022700000260546009601960296039600681A49C4
:1022800088422ED11949C86940F00050C861C86918
:1022900000F000500490886940F00400886188696B
:1022A000202700F0040004900320CDE90070694667
:1022B0000F4800F03DFB104C0E4820601020C4E990
:1022C00001068020E060400020618000E661C4E9F2
:1022D0000507204600F0F2F908B1FEF7E2FFEC60D6
:1022E000656205B0F0BD00000074004000100240BF
:1022F0000008014044040240EC2B002010B590F887
:1023000021100022022905D00421816380F82020B9
:10231000012010BD01680B6823F00E030B600168FB
:102320000B6823F001030B6090F84030C46B01216F
:1023300001FA03F3636080F8211080F82020104632
:1023400010BD00002DE9F05F90F821100024022953
:1023500003D004218163012485E001680A6822F02A
:102360000E020A6001680A6822F001020A603F4E0C
:102370003E4FB215DFF8F4C0DFF8F090DFF8ECA0C4
:10238000DFF8E8B0DFF8E4E00168783F13011502F8
:10239000ACF1640CA9F15009AAF13C0AABF1280B8D
:1023A000AEF1140E4FF48018B14227D9B9420ED0C5
:1023B000614512D049451DD0514518D0594518D016
:1023C000714501D1424615E0294EB14201D10122A9
:1023D00010E0274E1436B14201D110220AE0244EFB
:1023E0002836B14206D0224A3C32914201D11A46E7
:1023F00000E02A461E49091F0A602BE0B94213D0AB
:10240000614517D0494522D051451DD059451DD0B1
:10241000714501D142461AE0B14202D14FF08072BB
:1024200015E0134EB14201D1012210E0104E1436D6
:10243000B14201D110220AE00D4E2836B14206D039
:102440000B4A3C32914201D11A4600E02A46074924
:1024500080394A60012180F82110002180F8201085
:10246000416B01B188472046BDE8F09F80000240E3
:10247000080402402DE9F05FC16B0A6801680B682F
:10248000046C4FF0040808FA04F8844D844E854F1C
:10249000DFF814C2DFF81492DFF814A2DFF814B2E8
:1024A000DFF814E218EA020F65D05FEA437862D5DC
:1024B0000A68920603D40A6822F004020A60DFF870
:1024C000F0814FF48062016808F1140813011402CE
:1024D000414524D9A9420DD0B1420FD0B9421AD0FA
:1024E000614515D0494515D0514501D1120312E07F
:1024F000594501D104220EE0714501D140220AE084
:102500006D4D1435A94206D06B4A2832914201D153
:102510001A4600E022466749091F0A6029E0A942DD
:1025200013D0B14215D0B94220D061451BD04945E6
:102530001BD0514502D14FF4800217E0414502D132
:102540004FF0806212E0594501D104220EE071453E
:1025500001D140220AE0584D1435A94206D0564A0E
:102560002832914201D11A4600E022464B490839EF
:102570004A60C16A71E04FF0020808FA04F818EAEC
:10258000020F70D05FEA83786DD50A68920606D490
:102590000A6822F00A020A60012180F82110DFF89F
:1025A00010814FF40072016808F11408130114023D
:1025B000414524D9A9420DD0B1420FD0B9421AD019
:1025C000614515D0494515D0514501D1120312E09E
:1025D000594501D102220EE0714501D120220AE0C5
:1025E000354D1435A94206D0334A2832914201D1E3
:1025F0001A4600E022462F49091F0A6029E0A94235
:1026000013D0B14215D0B94220D061451BD0494505
:102610001BD0514502D14FF4001217E0414502D1C1
:102620004FF0007212E0594501D102220EE07145CF
:1026300001D120220AE0204D1435A94206D01E4ABD
:102640002832914201D11A4600E022461349083946
:102650004A60002180F82010816A00291CD0BDE862
:10266000F05F0847FFE70825A540154214D01A0778
:1026700012D50A6822F00E020A6090F84020C36B5F
:10268000012101FA02F25A60816380F821100021D1
:1026900080F82010016BE0E7BDE8F09F08000240E1
:1026A0001C0002403000024044000240580002403A
:1026B0006C000240080402401C04024030B560B1C6
:1026C0001A4B026814219A4209D2194B1344B3FBE6
:1026D000F1F18900016417490AE0012030BD134B74
:1026E0005B421344B3FBF1F1890001640F490839DF
:1026F000C163022180F82110136843F6F0718B4307
:10270000F0E901142143D0E902452C432143046937
:102710002143446921438469214319431160002105
:102720004163012242770177084630BD0804024028
:10273000F8FFFDBF0000024070B5044690F820008D
:10274000002501280CD0012084F8200094F8216095
:102750000020012E06D084F820000225284670BDF6
:10276000022070BD022684F82160A06320680668FC
:1027700026F0010606602046FEF764FDE06A0028A8
:102780002068016802D041F00E0106E021F004014A
:1027900001602068016841F00A0101602068016859
:1027A00041F001010160D9E770B5044600F0CEF9AF
:1027B0000546601C02D004480078044400F0C6F9C5
:1027C000401BA042FAD370BD380A00202DE9F04723
:1027D000054626480F460126017E01290FD001211A
:1027E000814601762868DFF888804CF25034022850
:1027F00008D0A2462046FEF7B7FDA8B131E002207E
:10280000BDE8F0872046FEF7AFFD08BB0120FEF7CC
:102810004BFD2046FEF7A8FDD8F81010064621F023
:102820000401C8F810101CE04FF0FF303860AC68AD
:1028300011E02046FEF74AFD5046FEF795FDD8F818
:102840001010060021F00201C8F8101001D03C6001
:1028500007E004F50064D5E9020100EBC120A042C5
:10286000E7D8002189F818103046C9E748700020E1
:10287000002002400348016941F08001016100200D
:1028800070470000002002402DE9F05F07461C4819
:1028900088460024017E15461E46012909D00121E3
:1028A000814601764CF2503A5046FEF75DFD18B174
:1028B00022E00220BDE8F09F012F02D0022F00D0BD
:1028C0000427D346DFF83CA0220128463146FDF715
:1028D0009DFC81B208EB4400FEF70AFD5846FEF766
:1028E00043FDDAF8102022F00102CAF8102018B9CE
:1028F000641CE4B2BC42E7D3002289F81820D9E76F
:102900004870002000200240064900200A69120693
:1029100007D5054A4A60054A4A600969090600D593
:10292000012070470020024023016745AB89EFCDAD
:102930002DE9F84FDFF8C891002409F1040A0AF1E3
:10294000040B23460F270BF1040ED1E00125A5400F
:1029500006EA0502AA4276D1DFF8A8C14E68A6EBC6
:102960000C0866452BD00DDC032E34D005DC36B3C5
:10297000012E19D0022E2FD11BE0112E16D0122EAF
:102980002AD119E0B8F5881F19D006DCB8F5803FC8
:1029900015D0B8F5801F1FD111E0B8F5001F0ED07B
:1029A000B8F5041F18D10AE0CB6815E0CB681B1DF1
:1029B00012E0CB6808330FE0CB680C330CE08B6877
:1029C0002BB1012B4FF0080303D0456104E0042331
:1029D00002E0056100E00023FF2A01D8064601E07D
:1029E00000F104064FEA840501D9A5F12005D6F8C7
:1029F000008007FA05FC28EA0C0803FA05F548EA06
:102A00000508C6F800804D68ED0070D53E4DAE69F2
:102A100046F00106AE61AD6924F0030605F001053C
:102A200000953A4D06EB050CDCF80850A607360F6A
:102A300007FA06F825EA0805DFF8D480404503D1F7
:102A40004FF0000825E052E0DFF8C880404502D191
:102A50004FF001081DE0DFF8C080404502D14FF083
:102A6000020816E0DFF8B480404502D14FF00308B9
:102A70000FE0DFF8AC80404502D14FF0040808E0D9
:102A8000DFF8A080404502D14FF0050801E04FF08B
:102A9000060808FA06F848EA0508CCF808804D68E8
:102AA000D9F80060ED034D4601D5164300E096438A
:102AB0002E604D68DAF80060AD03554601D5164327
:102AC00000E096432E604D68DBF80060ED025D4645
:102AD00001D5164300E096432E604D68DEF8006095
:102AE000AD02754601D5164300E096432E60641C86
:102AF0000A681646E2407FF429AFBDE8F88F00006F
:102B000000040140000011100010024000000140CC
:102B100000080140000C0140001001400014014079
:102B200000180140001C01408068084000D00120CE
:102B30007047C26821EA02030A4043EA0241016188
:102B400070470AB1016170470904FBE701488068DA
:102B500070470000380A002002488168027811445A
:102B600081607047380A0020074810B5016841F0BD
:102B700010010160032000F095F8002000F006F835
:102B800000F03EF8002010BD0020024000B50146D4
:102B900087B000222C2000F065F82C2000F054F8BB
:102BA0001348816941F400518161806905A900F4ED
:102BB00000500690684600F01DF900F04BF90D49F1
:102BC0000D4AB0FBF1F10D48491E0260416040F230
:102BD000E7320021C0E90321816000F051FB10B110
:102BE000012007B000BD054800F098FBF9E70000A0
:102BF0000010024040420F0000340140402D0020F0
:102C00000F4808B5816941F001018161816901F0D6
:102C100001010091C16941F08051C161C069002288
:102C200000F0805000900F21901E00F01BF8054826
:102C3000416821F0E06141F00071416008BD000091
:102C40000010024000000140002809DB00F01F02D4
:102C5000012191404009800000F1E020C0F80011FE
:102C600070470000F0B40E4B1B680C46C3F3022300
:102C7000C3F10705042D00D90425191D072901D228
:102C8000002300E0DB1E012606FA05F1491E214063
:102C900099409E40761E16403143F0BC06F07CBD44
:102CA0000CED00E0064900F0070208684FF6FF034C
:102CB000184040EA0220034A1043086070470000B1
:102CC0000CED00E00000FA052DE9F0470F46050085
:102CD00061D0434E306800F00700B84209D2306836
:102CE00020F0070038433060306800F00700B84239
:102CF00051D128683B4C810712D5400703D5606845
:102D000040F4E06060602878000703D5606840F414
:102D1000605060606068A96820F0F000084360605F
:102D20002878C00728D06868012810D021680228B8
:102D300010D0890700292EDA616821F003010143D0
:102D40006160FFF703FF804641F288390DE021689A
:102D50008903EFE78901EDE7FFF7F8FEA0EB080133
:102D6000494502D90320BDE8F0876068696800F032
:102D70000C00B0EB810FEFD1306800F00700B842D3
:102D80000BD9306820F0070038433060306800F01D
:102D90000700B84201D00120E5E72878400705D5B3
:102DA0006068E96820F4E060084360602878000704
:102DB00006D56068296920F4605040EAC10060606F
:102DC00000F058F86168084AC1F30311515CC8402B
:102DD0000649086006480068FFF7D8FE0020C2E7F1
:102DE0000020024000100240C0CA0008340A00203F
:102DF0003C0A00200F2202600C4A536803F00303D0
:102E00004360536803F0F0038360536803F4E063A6
:102E1000C36052684FF4E06303EAD20202610448DF
:102E2000006800F0070008607047000000100240D2
:102E3000002002400448054900684968044AC1F37B
:102E40000221515CC8407047340A00200010024043
:102E5000D0CA00080448054900684968044AC1F31B
:102E6000C221515CC8407047340A00200010024063
:102E7000D0CA000812A185B00FC98DE80F0014A0B8
:102E8000144A006804905168134801F00C03042BA5
:102E900010D0082B0ED1C1F38343C9031DF80300E2
:102EA0000AD5516804AAC1F34041515C0A4A504313
:102EB000B0FBF1F005B0704708494843FAE700005D
:102EC00002030405060708090A0B0C0D0E0F10106B
:102ED000010200000010024000127A0000093D00CB
:102EE0002DE9F84F040070D02078C04DC00749D0BC
:102EF0006868C0F38100012807D06868C0F38100CA
:102F0000022809D16868C00306D52868800339D52E
:102F100060680028E7D035E06068B0F5803F0BD0EE
:102F200010B1B0F5A02F11D0286820F480302860AF
:102F3000286820F4802002E0286840F4803028606F
:102F4000606890B1FFF702FE06460AE0286840F488
:102F500080202860F0E700BFFFF7F8FD801B6428A1
:102F600073D828688003F7D50CE0FFF7EFFD06461D
:102F700005E000BFFFF7EAFD801B6428F0D8286851
:102F80008003F7D420789A4E80074FF001094FF064
:102F9000000839D5686810F00C0F07D06868C0F3D6
:102FA0008100022809D16868C00306D42868800718
:102FB00014D52069012808D110E02069B0B1C6F805
:102FC0000090FFF7C3FD074605E00AE1FFF7BEFDED
:102FD000C01B0228C4D828688007F7D52868616913
:102FE00020F0F80040EAC10028600DE0C6F800803B
:102FF000FFF7ACFD074604E0FFF7A8FDC01B022861
:1030000023D828688007F7D4207800072CD5794882
:10301000A169D9B1C0F80090FFF798FD074604E018
:10302000FFF794FDC01B02280FD8686A8007F7D508
:1030300071484FF4FA510068B0FBF1F0009000BF06
:103040000098411E0091FAD20EE080E0C0F80080A6
:10305000FFF77CFD074604E0FFF778FDC01B022860
:1030600075D8686A8007F7D42078400760D5E8698A
:103070000027C00008D4E86940F08050E861E869A2
:10308000012700F0805000905C480168C90513D406
:103090000168834641F480710160FFF757FD824665
:1030A00006E000BFFFF752FDA0EB0A0064284ED8EF
:1030B000DBF80000C005F5D5E06801280AD008B1AA
:1030C000052813D0286A20F001002862286A20F021
:1030D000040002E0286A40F001002862E06841F242
:1030E000883B98B1FFF732FD82460BE0286A40F03A
:1030F00004002862EEE700BFFFF728FDA0EB0A01FD
:1031000059455AD8286A8007F6D50CE0FFF71EFD0E
:10311000824605E0FFF71AFDA0EB0A0159454CD89D
:10312000286A8007F6D41FB1E86920F08050E86172
:10313000E06988B36968C1F38101022944D002289B
:10314000C6F8608004D0FFF701FD044638E034E0A3
:10315000FFF7FCFC074604E0FFF7F8FCC01B022861
:103160002BD828688001F7D4206AB0F5803F05D1BC
:103170006868A16820F4003008436860D4E9080159
:103180000843696821F4741108436860C6F86090C8
:10319000FFF7DCFC044606E025E000BFFFF7D6FCA5
:1031A000001B022809D828688001F7D51BE000BF62
:1031B000FFF7CCFC001B022802D90320BDE8F88FE2
:1031C00028688001F4D40EE00128F7D06868226AEC
:1031D00000F48031914204D1616A00F47010884299
:1031E00001D00120EAE70020E8E7000000100240DB
:1031F0000000424280044242340A00200070004035
:103200007047704770B590F83C20012A2CD00124FB
:1032100080F83C40022280F83D2003685A689D688F
:1032200022F070060A6832435A60104B02689A42D4
:103230000ED00F4B9A420BD0B2F1804F08D00D4BFD
:103240009A4205D00C4B9A4202D00C4B9A4204D1C0
:10325000496825F080031943916080F83D400021C2
:1032600080F83C10084670BD022070BD002C014063
:10327000003401400004004000080040000C004001
:1032800010B5040003D094F83D0010B107E0012010
:1032900010BD002084F83C00204600F01FF80220FA
:1032A00084F83D00211D206805F0BAFD012084F856
:1032B000460084F83E0084F83F0084F8400084F81B
:1032C000410084F8420084F8430084F8440084F804
:1032D000450084F83D00002010BD000008B50C4AF0
:1032E00001680C48914207D1816941F40061816114
:1032F000806900F4006009E0074A914207D1C16982
:1033000041F00401C161C06900F00400009008BDF3
:10331000002C0140001002400008004090F83D10D1
:10332000012901D001207047022180F83D10016879
:10333000CA6842F00102CA6000680E4988420ED095
:103340000D4988420BD0B0F1804F08D00B4988421C
:1033500005D00B49884202D00A49884204D18168CD
:1033600001F00701062903D0016841F00101016065
:1033700000207047002C0140003401400004004050
:1033800000080040000C004070B5044690F83C0076
:10339000012817D0012584F83C50022084F83D0014
:1033A0002068826822F0770222F47F4282600868F7
:1033B000502830D00DDC20284DD005DC98B31028E3
:1033C0003BD148E0022070BD302844D0402834D1A1
:1033D00039E0602828D0702806D0B0F5805F2CD066
:1033E000B0F5005F29D10AE0CB68D1E9012120685E
:1033F00005F05CFD2068816841F0770109E0CB6849
:10340000D1E90121206805F051FD2068816841F46F
:103410008041816011E0CA684968206805F058FD64
:103420005021206807E016E0CA684968206805F066
:1034300060FD6021206805F043FD84F83D500020C8
:1034400084F83C0070BDCA684968206805F040FDFA
:1034500040212068EFE7226801461046EBE77047FD
:1034600070B50446006801694FF00005C94389073B
:1034700015D4C168C943890711D4E91E016101202F
:103480002077206880698007204602D0FFF7E7FF99
:1034900004E000F098F8204600F096F825772068C0
:1034A0000169C943490717D4C168C943490713D4FF
:1034B0006FF004010161022020772068806910F418
:1034C000407F204602D0FFF7CAFF04E000F07BF8FF
:1034D000204600F079F8257720680169C94309077B
:1034E00016D4C168C943090712D46FF008010161FD
:1034F000042020772068C0698007204602D0FFF7AB
:10350000AEFF04E000F05FF8204600F05DF825779C
:1035100020680169C943C90617D4C168C943C906EF
:1035200013D46FF010010161082020772068C06972
:1035300010F4407F204602D0FFF791FF04E000F036
:1035400042F8204600F040F8257720680169C94319
:10355000C90708D1C168C943C90704D1891E0161DF
:10356000204600F033F820680169C943090609D4F0
:10357000C168C943090605D46FF080010161204686
:10358000FFF73EFE20680169C943490609D4C168B6
:10359000C943490605D46FF040010161204600F09F
:1035A0001FF820680169C94389060BD4C168C94363
:1035B000890607D46FF0200101612046BDE8704004
:1035C000FFF71FBE70BD70477047000000680349D9
:1035D000884201D1FFF7C0BA7047000000340140B3
:1035E000704710B504460068416994F83920C1F36A
:1035F000C011212A0BD151B1416921F080014161F3
:10360000206B08B1FEF77AFE204605F0C5FD206864
:10361000416994F83A20C1F38011222A0BD151B1AB
:10362000416921F040014161606B08B1FEF766FE1F
:10363000204605F0A3FD002010BD704770B502685C
:1036400004461068D168536910F00F0F52D003F090
:10365000010501F490762E435FD0C20705D0CA055C
:1036600003D5E26B42F00102E263420705D5DA07B7
:1036700003D0E26B42F00202E263820705D5DA076B
:1036800003D0E26B42F00402E263020707D501F0C7
:1036900020022A4303D0E26B42F00802E263E26BAD
:1036A000002A33D0800604D5880602D5204605F0CE
:1036B0007CFD20684069E16BC0F38010090700D4ED
:1036C00028B3204605F05AFD2068416949061AD5FD
:1036D000416921F040014161606BA0B11B49416328
:1036E000606BFEF72FFE002810D0606B416BBDE8C9
:1036F00070400847830610D58B060ED52046BDE8DE
:10370000704005F052BD2046FFF797FF70BD204680
:10371000FFF793FF0020E06370BD030606D50B069C
:1037200004D52046BDE8704005F0E2BD4006F3D563
:103730004806F1D5D168204621F04001D160202112
:1037400084F8391000F010FA70BD0000DD90000818
:1037500070B5040004D094F83900002510B106E0DB
:10376000012070BD84F83850204600F023F8242052
:1037700084F839002068C16821F40051C1602046F6
:1037800005F05AFD2068016921F49041016120682B
:10379000416921F02A0141612068C16841F400516A
:1037A000C160E563202084F8390084F83A000020E5
:1037B00070BD00002DE9F04F85B000250095019502
:1037C000029503950446774E036877480221032249
:1037D0004FF00408B34229D1C36943F48013C36195
:1037E000C36903F480130493836943F01003836176
:1037F000836903F010030493836943F0200383611A
:103800008069039200F020000490C802CDE9000115
:1038100069466648FFF78CF8CDE90085694664483B
:103820000295FFF785F805B0BDE8F08FDFF884C199
:10383000614F80264FF480694FF0200A4FF4005BFF
:10384000634544D1836943F480438361836903F40E
:1038500080430493836943F0040383618069039286
:1038600000F004000490B000CDE90001694638463C
:10387000FFF75EF8CDE90095694638460295FFF7F7
:1038800057F84F4F4D4807F11403C7E90005C7E942
:1038900002563D6183E8200C3846FEF70FFF08B161
:1038A000FDF7FFFC67637C624448464F143801C74C
:1038B000102061C7434847F810597D61BD61FD6123
:1038C000FEF7FCFE08B1FDF7ECFC276333E0DFF800
:1038D000F8C0634531D1C36943F40033C361C369A0
:1038E00003F400330493836943F004038361806924
:1038F000CDE9008100F00400CDE903206946384697
:10390000FFF716F80820CDE900056946384602950C
:10391000FFF70EF82D4F294807F114031430C7E9BB
:103920000005C7E902563D6183E8200C384633E0C4
:10393000FDF7B7FC34E07C6275E7254FBB42FBD155
:10394000C36943F48023C361C36903F480230493F0
:10395000836943F0080383618069CDE9009100F039
:103960000800CDE903201B4F69463846FEF7E0FF0B
:10397000F814CDE90005694638460295FEF7D8FFF0
:103980000E48154F2838C7E90005C7E902563D61C2
:103990007D61BD613846FD61FEF790FE0028C7D10C
:1039A0006763C8E70050004000100240001001406B
:1039B0000014014000380140000801405800024056
:1039C000302C0020742C002000440040B82C002033
:1039D00000480040000C0140FC2C0020F8B50446D3
:1039E00090F83A0020283CD1C1B3BAB394F838001B
:1039F000012836D0012084F83800A162A285002574
:103A0000E563222084F83A00636B17489862636B81
:103A10001648D862636B16481863606B134645639B
:103A20000846666B216802463046091DFEF784FE93
:103A3000206801684168009184F83850C16841F4F9
:103A40008071C1602068416941F0010141612068D5
:103A5000416941F0400141610020F8BDFFE70120CC
:103A6000FBE70220F9E70000379100087391000896
:103A7000ED900008704770472DE9F843044690F830
:103A800039001F4616460D4620284CD1C5B1BEB19F
:103A900094F83800012846D0012084F838004FF00F
:103AA0000008C4F83C80212084F83900FFF74EF864
:103AB000A6848146E684A068B0F5805F03D004E068
:103AC0000120BDE8F883206928B12E465FF000058B
:103AD00084F838800EE00026FAE78021204605F0C1
:103AE0003AFCA0B9AEB116F8010B21684860E08C31
:103AF000401EE084E08C4B464FF000020097002807
:103B0000EBD14FF04001204605F025FC30B10320F9
:103B1000D7E735F8020BC0F30800E6E7202084F869
:103B200039000020CDE70220CBE790F83930202B78
:103B300018D1A9B1A2B190F83830012B12D001628E
:103B40008284C2840021C163212280F8392080F858
:103B500038100068C16841F08001C16000207047E2
:103B6000012070470220704770470000154810B5CB
:103B7000418811B9017D062901D0002010BD012125
:103B8000104C4180463C807F2070062060700020F1
:103B9000A070A520E07020716071A071E0712072AA
:103BA0006072A072E072207360730E21204600F0F4
:103BB00007F9010AA1730449E0731020088001206D
:103BC00010BD0000A4370020C40900202DE9F041F9
:103BD0008AB007462B4E2C4C28216846FCF745FB43
:103BE00000206D4605E02118497F25F81010401C83
:103BF000C0B2217E8142F6D8207DDFF89080062871
:103C000004D1012241462846FDF7E6FB0122414648
:103C10006846FDF7D3FBBDF800003874BDF800001E
:103C2000052800D2F080207DDFF86480062804D1CA
:103C300008224146A81CFDF7CFFB08224146A81CDC
:103C4000FDF7BCFB002013E005EB40022318518870
:103C50009B7F994202D0237D062B10D0082905D2E4
:103C600006EB4003998491783A185174401CC0B215
:103C7000217E8142E8D801200AB0BDE8F081002011
:103C8000FAE70000A8360020A437002030F007082B
:103C900040E0070870B51548418811B9017D062933
:103CA00001D0002070BD114C01214180463C817F34
:103CB0002170062161701025A57090F82000E07039
:103CC000A52020716071A071E07120726072A072F5
:103CD000E072207360730E21204600F071F8010A33
:103CE000A173E07302480580012070BDA437002055
:103CF000C4090020164810B5418811B9017D062974
:103D000001D0002010BD124C01214180463C817F32
:103D10002170062161701221A17090F82000E070DE
:103D2000A52020716071A071E07120726072A07294
:103D3000E072207360730E21204600F041F8010A02
:103D4000A1730449E07310200880012010BD000019
:103D5000A4370020C4090020164810B5418811B9C5
:103D6000017D062901D0002010BD124C01214180A7
:103D7000463C817F2170062161701421A170C17FB2
:103D8000E17090F820002071A5206071A071E071B1
:103D900020726072A072E072207360730E21204660
:103DA00000F00EF8010AA1730349E07310200880A7
:103DB000012010BDA4370020C4090020FEE7000048
:103DC00070B50A4DFF22134605F5807606E000BF68
:103DD00010F8014B54402A5D5A40335D491E89B2A8
:103DE000F6D203EB022080B270BD000090BD000847
:103DF000002203E0491E00F8012B89B20029F9D105
:103E000070470000F0B58BB00546344C344E282185
:103E10006846FCF72AFAB4F81D00324F40BAADF8F4
:103E20000000B4F81F0040BAADF80200B4F8210059
:103E300040BAADF80400B4F8230040BAADF806006B
:103E4000207D062804D1042239466846FDF7C4FACD
:103E5000042239466846FDF7B1FABDF80000020AAF
:103E60002A74BDF80000C0B26874BDF80210090AD7
:103E7000A974BDF80210E974BDF80410090A297587
:103E8000BDF804106975BDF80610090AA975BDF8DA
:103E90000810E975617F8A4205D1A27F904202D164
:103EA000207D062802D000200BB0F0BD0E48C17066
:103EB000827014F81F1F4170617801700168F1640D
:103EC00000BFA178C170E17881702179417061797A
:103ED00001700068706700BF0120E5E7A43700208B
:103EE000A03E002000C0070828030020F0B58BB0DA
:103EF00005461C4E1C4C28216846FCF7B6F9B4F860
:103F00001D001A4F40BAADF80000207D062804D1EC
:103F1000012239466846FDF75FFA012239466846B4
:103F2000FDF74CFABDF80000000A2874BDF8000047
:103F30006874BDF80000A0F57F41FF3901D0A6F8F4
:103F40006400287C617F884206D1687CA17F88421A
:103F500002D1207D062802D000200BB0F0BD012048
:103F6000FBE70000A8360020A437002040F0070837
:103F70007CB50C460546082210316846FDF778F9F5
:103F8000208AC0F3C500382802D2C0F1380201E00F
:103F9000C0F178020949204600F094FB08226946E6
:103FA000204600F08FFB102221462846FDF760F9DD
:103FB00058220021204600F0C6FB7CBDF4090020F9
:103FC00000214161016105490160054941600349E2
:103FD000C94381600249C943C160704701234567F5
:103FE00089ABCDEF2DE9F04F50F804BB002590E8E8
:103FF000580091B0EA464FF040092A46001F8F183A
:10400000121D97F80280B7F800C0FF7868F31F4CC4
:104010004CEA076C4AF825C06D1C4A45EFD303EA09
:10402000040126EA03021143FE4A009D0A4405EBFF
:104030000B01114403EB716202EA030124EA020757
:104040003943F94F3944019F3E44314402EB315129
:1040500001EA020623EA01073E43F44F3E44029F71
:104060003C44344401EBF43404EA010622EA040738
:104070003E43EF4F3E44039F3B44334404EBB323A2
:1040800003EA040621EA03073E43EA4F3E44049F45
:104090003A44324403EB726202EA030624EA02075E
:1040A0003E43E54F3E44059F3944314402EB3151D4
:1040B00001EA020623EA01073E43E04F3E44069F21
:1040C0003C44344401EBF43404EA010622EA0407D8
:1040D0003E43DB4F3E44079F3B44334404EBB32352
:1040E00003EA040621EA03073E43D64F3E44089FF5
:1040F0003A44324403EB726202EA030624EA0207FE
:104100003E43D14F3E44099F3944314402EB315183
:1041100001EA020623EA01073E430A9FA6F5244668
:104120003C444F3E344401EBF43404EA010622EAF5
:1041300004073E43C54F3E440B9F3B44334404EBCE
:10414000B32303EA040621EA03073E43C04F3E447B
:104150000C9F3A44324403EB726202EA030624EAFB
:1041600002073E43BB4F3E440D9F3944314402EBAE
:10417000315101EA020623EA01073E43B64F3E44AD
:104180000E9F3C44344401EBF43404EA010622EA75
:1041900004073E43B14F3E440F9F3B44334404EB7E
:1041A000B32303EA010624EA01073E43AC4F3E4431
:1041B000019F3A44324403EBF26202EA040623EA26
:1041C00004073E43A74F3E44069F3944314402EB67
:1041D000F15101EA030622EA03073E43A24F2B44B2
:1041E0003E440B9F3C44344401EBB44404EA0206D1
:1041F00021EA02073E439D4F3E44334404EB3333F0
:1042000003EA010624EA01073E43994F3E44059F15
:104210003A44324403EBF26202EA040623EA04075A
:104220003E43944F3E440A9F3944314402EBF151DE
:1042300001EA030622EA03073E438F4F3E440F9FE5
:104240003C44344401EBB44404EA020621EA020788
:104250003E438A4F3E44049F3B44334404EB333394
:1042600003EA010624EA01073E43854F3E44099FC5
:104270003A44324403EBF26202EA040623EA0407FA
:104280003E43804F3E440E9F3944314402EBF15689
:1042900006EA030122EA030739437B4F3944039FAF
:1042A0003C44214406EBB14101EA020426EA02073C
:1042B0003C43764F3C44089F3B44234401EB33335B
:1042C00003EA060421EA06073C43714F3C440D9F74
:1042D0003A44224403EBF26202EA010423EA0107B2
:1042E0003C436C4F3C44029F3E44344402EBF45444
:1042F00004EA030622EA03073E43674F3E44079F52
:104300003944314404EBB14101EA020624EA0207D0
:104310003E43624F3E440C9F3B443344059E01EBB9
:104320003333164483EA01025D4F62403A4432441B
:10433000089E03EB3272264482EA0304594F4C4034
:104340003C4434440B9E02EB74540E4484EA020154
:10435000554F5940394431440E9E04EB31411E44BF
:1043600081EA0403514F53403B443344019E01EB27
:104370007323164483EA01024D4F62403A443244AB
:10438000049E03EB3272264482EA0304494F4C40F8
:104390003C443444079E02EB74540E4484EA020108
:1043A000454F5940394431440A9E04EB31411E4483
:1043B00081EA0403414F53403B4433440D9E01EBDB
:1043C0007323164483EA01023D4F62403A4432446B
:1043D00003EB32722E1982EA03043A4F4C403C44FC
:1043E0003444039E02EB74540E4484EA0201364FB7
:1043F000594039443144069E04EB31411E4481EA60
:104400000403324F53403B443344099E01EB732372
:10441000164483EA01022E4F62403A44324403EBD1
:10442000327257E078A46AD756B7C7E8DB70202409
:10443000EECEBDC1AF0F7CF52AC68747134630A824
:10444000019546FDD8988069AFF7448BBED75C894B
:104450002211906B937198FD8E4379A62108B4497F
:1044600062251EF640B340C0515A5E26AAC7B6E97F
:104470005D102FD65314440281E6A1D8C8FBD3E7C0
:10448000E6CDE121D60737C3870DD5F4ED145A45A3
:1044900005E9E3A9F8A3EFFCD9026F678A4C2A8DDE
:1044A0004239FAFF81F6718722619D6D0C38E5FD76
:1044B00044EABEA4A9CFDE4B604BBBF670BCBFBEC6
:1044C000C67E9B28FA27A1EA8530EFD4051D880413
:1044D00039D0D4D90C9E684F264482EA03044C405C
:1044E0003C4434440F9E02EB74540E4484EA0201AF
:1044F000624F594039443144029E04EB31411E441D
:1045000081EA04035E4F53403B44334401EB732381
:10451000154463EA04025B4E4A4032442A44079D34
:1045200003EBB262254462EA0104574E5C40344416
:104530002C440E9D02EBB4540D4464EA0301534E27
:10454000514031442944059D04EB71411D4461EA09
:1045500002034F4E634033442B440C9D01EBF32385
:10456000154463EA04024B4E4A4032442A44039DF8
:1045700003EBB262254462EA0104474E5C403444D6
:104580002C440A9D02EBB4540D4464EA03015140EB
:10459000424E31442944019D04EB71411D4461EABE
:1045A00002033F4E634033442B44089D01EBF32349
:1045B000154463EA04023B4E4A4032442A440F9DAC
:1045C00003EBB262254462EA0104374E5C40344496
:1045D0002C44069D02EBB4540D4464EA0301334EAF
:1045E0005140314429440D9D04EB71411D4461EA61
:1045F00002032F4E634033442B44049D01EBF3230D
:10460000154463EA04022B4E4A4032442A4403EB29
:10461000B2650B9A284E144465EA01025A403244AE
:104620002244029C05EBB2520C4462EA0301234E81
:10463000694031442144099C02EB71411C4461EA08
:1046400005031F4E534033442344046801EBF32316
:104650002C440460446823444360836819448160A7
:10466000C1681144C16040220021504600F06BF83F
:1046700011B0BDE8F08F0000E599DBE6F87CA21FE1
:104680006556ACC4442229F497FF2A43A72394AB70
:1046900039A093FCC3595B6592CC0C8F7DF4EFFF7E
:1046A000D15D84854F7EA86FE0E62CFE144301A304
:1046B000A111084E827E53F735F23ABDBBD2D72AFC
:1046C00091D386EB2DE9F0410F4601690546164668
:1046D000C1F3C50001EBC6012961B1EBC60F6969E1
:1046E00001D2491C696101EB5671C0F14004696156
:1046F000A64216D3284422463946183000F01AF84C
:1047000005F118012846FFF76DFC04E03919284629
:10471000FFF768FC403404F13F00B042F6D30020BC
:1047200000E00024321B39192844BDE8F04118305C
:10473000AFF3008010B5002302E0CC5CC4545B1CD6
:104740009342FAD310BD0023C9B201E0C1545B1CEF
:104750009342FBD3704770B5017845780846FBF764
:1047600065FD3038C4B2092C01D9E41FE4B22846F3
:10477000FBF75CFD3038C0B2092801D9C01FC0B2B8
:1047800000EB0410C0B270BD2DE9F04F85B00024DD
:104790003B480094019402940394816941F0200104
:1047A0008161816901F020010491816941F0040176
:1047B0008161816901F004010491816941F008017E
:1047C0008161816901F008010491816941F0100162
:1047D00081618069DFF8AC9000F010000490002245
:1047E00013214846FEF7ADF9DFF89CA04FF440577F
:1047F000002239465046FEF7A4F9DFF890B04FF496
:104800008068002241465846FEF79BF91320012597
:104810000226CDE90005CDE9024669464846FEF785
:1048200087F800970396CDE9015469465046FEF794
:104830007FF8B800CDE90004694650460294FEF7BF
:1048400077F84FF47070CDE9000469465846029439
:10485000FEF76EF84FF41060CDE900046946484653
:104860000294FEF765F8CDF800800396CDE9015477
:1048700069465846FEF75CF805B0BDE8F08F0000C9
:104880000010024000080140000C014000100140EF
:1048900010B5002205212720FEF7E4F92720FEF7B6
:1048A000D3F9002205212520FEF7DCF92520FEF7AB
:1048B000CBF9002205212620FEF7D4F92620FEF7A9
:1048C000C3F9002205211E20FEF7CCF91E20FEF7B9
:1048D000BBF9002205211920FEF7C4F91920FEF7C3
:1048E000B3F9002205211020FEF7BCF91020FEF7D5
:1048F000ABF9002205210F20FEF7B4F90F20FEF7D7
:10490000A3F9002205210D20FEF7ACF9BDE8104007
:104910000D20FEF799B9000010B586B000241848A4
:104920000094019402940394049414490594C0E9FA
:1049300000144FF6FF71C0E902414FF40071C0E965
:1049400004148461FEF79CFC08B172B6FEE74FF4D4
:104950008050009069460A48FEF716FD08B172B60D
:10496000FEE7049404A906480594FEF74BFC0028D2
:1049700001D072B6FEE706B010BD0000002C014069
:104980005C29002010B586B00024164800940194DC
:1049900002940394049412490594C0E900144FF65C
:1049A000FF71C0E9024104618461FEF769FC08B14E
:1049B00072B6FEE74FF48050009069460948FEF752
:1049C000E3FC08B172B6FEE7049404A90548059417
:1049D000FEF718FC002801D072B6FEE706B010BD45
:1049E00000080040A429002010B5114C0F480C21EC
:1049F00020604FF4165060600020A060E060C4E9C1
:104A00000401A061E0612046FEF7A2FE08B172B683
:104A1000FEE72068C16841F01001C160BDE81040A8
:104A20004FF4807203490248FEF7D8BF00380140B6
:104A30002C2A0020BC0C002010B5114C0F480C2172
:104A400020604FF4164060600020A060E060C4E980
:104A50000401A061E0612046FEF77AFE08B172B65B
:104A6000FEE72068C16841F01001C160BDE8104058
:104A70004FF4806203490248FEF7B0BF0044004093
:104A80006C2A00200020002010B5114C0F480C218A
:104A900020604FF4165060600020A060E060C4E920
:104AA0000401A061E0612046FEF752FE08B172B633
:104AB000FEE72068C16841F01001C160BDE8104008
:104AC0004FF4807203490248FEF788BF0048004057
:104AD000AC2A0020BC0D0020FEE7FEE72DE9F04FD8
:104AE000FE4D002087B04FF4007205F58066014648
:104AF00025F8101026F81010401C9042F8DBDFF863
:104B0000E0B3DFF8E0A389469BF806209BF8053068
:104B10000DF1080802EB0322AAF804209BF80820F4
:104B20009BF807304FF4806702EB0322AAF80620B7
:104B3000ED4A9BF8043014688AF800301160EBA14C
:104B4000EC4BD1E90001CDE900010FCB88E80F0063
:104B50003946E948FDF7EDFF9AF80000DFF89C833D
:104B600001282CD002287DD003287CD15E468521E7
:104B7000301DFFF725F93119AAF80E0011F8062D9E
:104B80005546497802EB012189B2AAF80C108842F7
:104B90006AD10022102144464046FDF7D2FF502042
:104BA00004F0D2FFAB8802AAD5A1584604F0E0FD7C
:104BB00082B25946D448FEF7B8FFD34DB5E1BAF8F2
:104BC000041001297DD19BF84C109BF849209BF8DB
:104BD0004B3001EB02619BF84A205E46120402EB67
:104BE00003221144CAF810108521301DFFF7E8F8A0
:104BF0003119AAF80A0011F8062D497802EB0121B3
:104C000089B28842AAF80C104FF000006CD1BF495D
:104C1000331842185B7A92F87E209A4203D1401CE6
:104C20005828F5DB2BE0582829DA002006EB400154
:104C3000B1F8091025F81010401C2C28F6DBAE4CFA
:104C400039462046FDF775FFB0492C227E31A34836
:104C5000FCF7C2FB39462046FDF76BFF502004F0FD
:104C600073FF02E064E060E043E0AAF80890A8481F
:104C7000CAF8140039462046FDF75BFF06E0BAF893
:104C80000800012802D9401EAAF808000020494661
:104C90003154401CB842FBDB5446BAF808209DA1B1
:104CA0008E4804F065FD6080002210214546404694
:104CB000FDF747FF502004F047FF6288874992487C
:104CC00000E031E0FEF731FF8F4C02E0012005F0FB
:104CD0003FFA94F839002128F8D0502004F034FF2E
:104CE000502004F031FFD9E049463154401CB8420D
:104CF000FBDB0022102144464046FDF722FF5020F6
:104D000004F022FF6846FBF7BBFA82B264236946CF
:104D10007D48FEF7B1FE502004F016FF012210215D
:104D20002046FDF70EFF00BF00BF07B0BDE8F08FC3
:104D3000A4F10A0081B20BF10400FFF741F80BEB7C
:104D40000403AAF80A0013F8062D51465B7802EB1B
:104D500003239BB2AAF80C3098427DD10889B1F8A0
:104D600004C00346401C604501D0634574D16045D2
:104D700061D1A4F10F0000EBD07121F00103984242
:104D80004FF0000001D15A460FE0A4F11001DC46BB
:104D900001EBD17119E000BF02EB4003B3F8093019
:104DA00025F8103026F81030401CB0EB610FF3DB13
:104DB000C1F34F061BE000BF0CEB4003B3F8093012
:104DC00025F8103026F81030401CB0EB610FF3DBF3
:104DD00021F0010110024853885339464648FDF737
:104DE000A8FEA4F10E0000EBD070C0F34F063246CF
:104DF00055463A48DAF81410FCF7EEFA39463E48C0
:104E0000FDF797FE324646486969FCF7D7FA3946FE
:104E10003948FDF78EFEDAF8141021440F39CAF82C
:104E200014100A68CAF81C200968CAF8201039460C
:104E30003148FDF77EFE5446D4E90701884206D189
:104E400000BF39462C48FDF774FEA0882081002061
:104E500049465A46115400E027E0401CB842F9DBAD
:104E6000A38802AA26A11E4804F082FC0446002260
:104E7000102145464046FDF764FE502004F064FED4
:104E8000A2B217492048FEF750FE1F4C02E0012055
:104E900005F05EF994F839002128F8D0012210219C
:104EA0004FEA0500FDF74DFE3EE700221021444683
:104EB0004046FDF746FE502004F046FE6846FBF7EC
:104EC000DFF982B2642369460F48FEF7D5FD502012
:104ED00004F03AFE012210212046E3E74260002060
:104EE00000240020CC090020140300206572726F9A
:104EF000720D0A00B0CA000800100140000801400D
:104F000025733D25640D0A006C2A002000F0070877
:104F10000000040866696C653D25640D0A00000008
:104F200042640020012005F013F995F8390021288A
:104F3000F8D0012210212046FDF703FE00BF02F049
:104F400071FB00002DE9F0413B4D8AB0A5F58C675F
:104F5000A5F50E640026082238496846FCF72EFAAB
:104F600068464FF6FF7808E030F81610414502D049
:104F700005EB46029186761CF6B22988B142F3D839
:104F800001222F49FCF71AFABDF800004646B0424C
:104F900000D028812A49012238316846FCF70EFAF0
:104FA000BDF80000B0424FF000001FD14FF4617116
:104FB0000AE000BFC0EBC00202EB820207EB420234
:104FC000401CA2F84210C0B22A88521C8242F1D87A
:104FD00010E000BFC0EBC00202EB820207EB42020E
:104FE000BDF80010401CA2F84210C0B22988491C2C
:104FF0008142EFD800239846B3F10107A4F800805E
:10500000E780A7806680402104F10800FEF7F0FEEB
:105010005B1CDBB24834082BF0D30A4A00202B88F3
:10502000117802E00221401CC0B28342FAD811700C
:105030000AB0BDE8F0810000A836002020E0070893
:1050400020F0070820030020F0B585B00546184E73
:10505000184C14216846FBF708F9B4F81D00164FE8
:1050600040BAADF80000207D062804D1012239465F
:105070006846FCF7B1F90020ADF80000012239467E
:105080006846FCF79BF9BDF80000A6F84200000A4C
:105090002874BDF80010C9B26974627F904205D1CE
:1050A000A07F814202D1012005B0F0BD0020FBE7C6
:1050B00048320020A437002058F007082DE9F041BD
:1050C0008AB007462B4E2C4C28216846FBF7CDF8BA
:1050D00000206D4605E02118497F25F81010401C7E
:1050E000C0B2217E8142F6D8207DDFF8908006286C
:1050F00004D1012241462846FCF76EF901224146BF
:105100006846FCF75BF9BDF800003874BDF8000094
:10511000052800D23081207DDFF86480062804D184
:1051200008224146A81CFCF757F908224146A81C52
:10513000FCF744F9002013E005EB400223185188E6
:105140009B7F994202D0237D062B10D0082905D2DF
:1051500006EB4003998691783A185174401CC0B20E
:10516000217E8142E8D801200AB0BDE8F08100200C
:10517000FAE70000A8360020A437002020F0070836
:1051800020E007082DE9FC41184D00200090019017
:10519000298811B9297D062902D00020BDE8FC81AB
:1051A000124CAA7F8C3C062322706370A0701021E1
:1051B000E1702071FF2767718DF800208DF80130B4
:1051C0008DF802008DF804008DF8031001268DF88B
:1051D000057019466846FEF7F3FD010AA1710449FE
:1051E000E071082008802E800120D7E7A437002036
:1051F000C40900202DE9F0417E4904467B488E7F9A
:105200007B4A7D4D731E082B02D30020BDE8F08140
:105210002023E372897F02EBC6176174B7F87AE046
:1052200047217F22FF234FF0000CBEF1000F0FD06B
:10523000A174E274237584F815C0A175E275237614
:1052400084F819C0A176E276237784F81DC040E087
:10525000B7F900E04FEA1E6E84F812E0B7F900E0FB
:105260004FEA1E4E84F813E0B7F800E04FEA1E2E16
:1052700084F814E097F800E084F815E0B7F928E026
:105280004FEA1E6E84F816E0B7F928E04FEA1E4E8A
:1052900084F817E0B7F828E04FEA1E2E84F818E0EB
:1052A00097F828E084F819E0B7F950E04FEA1E6E4D
:1052B00084F81AE0B7F950E04FEA1E4E84F81BE07C
:1052C000B7F850E04FEA1E2E84F81CE097F85070B3
:1052D0006777B0F87A70B7B1A177E27784F82030B9
:1052E00084F821C084F8221084F8232084F8243024
:1052F00084F825C084F8261084F8272084F8283004
:1053000084F829C033E0B0F900703F0EA777B0F9F8
:1053100000703F0CE77707883F0A84F8207010F888
:10532000287B84F8217030F9287B3F0E84F82270A6
:1053300030F9287C3F0C84F8237030F8287C3F0A31
:1053400084F8247010F8287C84F82570B0F9007077
:105350003F0E84F82670B0F900703F0C84F8277077
:1053600007883F0A84F82870007884F8290006EB43
:10537000860705EBC706F08B58B104F82A1F627048
:10538000A37084F803C021716271A37184F807C00F
:105390002AE055F83700FBF750F8000E04F82A0F02
:1053A00055F83700FBF749F8000C607055F83700E6
:1053B000FBF743F8000AA07055F83700FBF73DF8FB
:1053C000E070B069FBF739F8000E2071B069FBF7A7
:1053D00034F8000C6071B069FBF72FF8000AA07177
:1053E000B069FBF72AF8E07101200FE720410020A7
:1053F000A4410020A4370020A03E00202DE9FC5F3E
:105400000446D0480190D248012600900020DFF8E1
:105410003083CD4BCD4ADFF83CB30146814682460E
:1054200005462718401CC0B23D740428F9D306EB8A
:10543000C60000EB461003EB4007B87804F8140FE1
:1054400000206070A070E07097F840502571607186
:1054500006EB8605A07105EB8615E07112F8157054
:1054600027726072A07202EB4507E07297F828C0BD
:1054700084F80CC06073A073E07312F815202274D6
:105480006074A074E07497F8282022756075A07588
:10549000E07501EBC10000EB411003EB4000032578
:1054A000B0F89E00143C10B184F82C5004E0481C65
:1054B000FCF780FD84F82C0009EB091000EB40019B
:1054C0000BEB4100B0F8C41011B184F8305003E088
:1054D00090F8BE1084F83010CAEBCA0101EB8102CB
:1054E000009901EB4201B1F8802022B184F83450D8
:1054F00084F8385006E011F87A2F84F8342089783F
:1055000084F83810B0F8C41011B184F83C5003E0AE
:1055100090F8C00084F83C00002504F82D5F657009
:10552000A57025716571A57125726572A5722573C7
:105530006573A57325746574A57417F8280FE07456
:1055400025756575A5753878E07525766576A57637
:1055500000202D3C2118401CC0B281F84850202862
:10556000F8D3019806EB860100EBC107F88B40B138
:1055700084F8685084F8695084F86A5084F86B5055
:105580000BE0786884F86800010A84F86910010C5F
:1055900084F86A10000E84F86B00F88BDFF8B8917D
:1055A00040B184F86C5084F86D5084F86E5084F8E3
:1055B0006F5013E008EBC610B0F92A00FAF72FFF7E
:1055C0004946FAF7BCFE84F86C00010A84F86D10B5
:1055D000010C84F86E10000E84F86F00F88B40B157
:1055E00084F8705084F8715084F8725084F87350C5
:1055F00013E008EBC610B0F90200FAF710FF4946B5
:10560000FAF79DFE84F87000010A84F87110010C0D
:1056100084F87210000E84F87300F88B40B184F89F
:10562000745084F8755084F8765084F8775013E0FD
:1056300008EBC610B0F92A00FAF7F1FE4946FAF76E
:105640007EFE84F87400010A84F87510010C84F859
:105650007610000E84F87700F88B40B184F878500B
:1056600084F8795084F87A5084F87B5013E008EB82
:10567000C610B0F95200FAF7D2FE4946FAF75FFEBB
:1056800084F87800010A84F87910010C84F87A1003
:10569000000E84F87B00F88B58B1762084F87C00EB
:1056A0007F2084F87D00FF2084F87E0084F87F50FE
:1056B0000BE0B86984F87C00010A84F87D10010CC5
:1056C00084F87E10000E84F87F00F88B84F88050F8
:1056D00084F8815084F8825084F88350F88B84F8E1
:1056E000845084F8855084F8865084F88750F88B6D
:1056F00084F8885084F8895084F88A5084F88B5054
:10570000F88B40B184F88C5084F88D5084F88E501A
:1057100084F88F500BE0B86984F88C00010A84F893
:105720008D10010C84F88E10000E84F88F00F88B19
:1057300004F8905F01206570A570E570BDE8FC9FDE
:10574000A4410020A03E0020A4490020C44E002017
:10575000483200203E380020CDCCCC3D2DE9F0432E
:10576000DFF814C30021A5224318491CC9B21A74DA
:105770000829F9D900210B4600EB8102491C137658
:1057800053769376C9B2D3760829F5D901217625C7
:105790007F264FF0FF0900BF01EB81040CEBC40230
:1057A000D78B57B101EB410404EBC10400EB840437
:1057B00023736373A373E37312E001EB410707EBF9
:1057C000C1075CF8344000EB87074FEA14283C73AC
:1057D00087F80D804FEA144887F80E80240EFC737A
:1057E000D48B54B101EB410404EBC10400EB8404FD
:1057F00023746374A374E37411E001EB410707EBB6
:10580000C10700EB870794683C744FEA142887F8B7
:1058100011804FEA144887F81280240EFC74D48B50
:1058200054B101EB410404EBC10400EB8404237583
:105830006375A375E37511E001EB410707EBC10741
:1058400000EB8707D4683C754FEA142887F8158069
:105850004FEA144887F81680240EFC75D48B54B197
:1058600001EB410404EBC10400EB8404237663766E
:10587000A376E37611E001EB410707EBC10700EBEC
:10588000870714693C764FEA142887F819804FEA95
:10589000144887F81A80240EFC76D48B54B101EB9F
:1058A000410404EBC10400EB840423776377A377FE
:1058B000E37711E001EB410707EBC10700EB870736
:1058C00054693C774FEA142887F81D804FEA144842
:1058D00087F81E80240EFC77D48B64B101EB410461
:1058E00004EBC10400EB840404F8205F667084F8C4
:1058F0000290E37012E001EB410707EBC10700EBF8
:105900008707946907F8204F4FEA142887F8018029
:105910004FEA144887F80280240EFC70D48B64B1DF
:1059200001EB410404EBC10400EB840404F8245FA0
:10593000667084F80290E37012E001EB410707EB18
:10594000C10700EB8707946907F8244F4FEA142832
:1059500087F801804FEA144887F80280240EFC7013
:10596000D48B64B101EB410404EBC10400EB84046B
:1059700004F8285F667084F80290E37012E001EB8F
:10598000410707EBC10700EB8707946907F8284F29
:105990004FEA142887F801804FEA144887F80280FC
:1059A000240EFC70D48B64B101EB410404EBC10400
:1059B00000EB840404F82C5F667084F80290E370B6
:1059C00012E001EB410707EBC10700EB8707946981
:1059D00007F82C4F4FEA142887F801804FEA144843
:1059E00087F80280240EFC70D48B64B101EB410473
:1059F00004EBC10400EB840404F8305F667084F8A3
:105A00000290E37012E001EB410707EBC10700EBE6
:105A10008707946907F8304F4FEA142887F8018008
:105A20004FEA144887F80280240EFC70D48B64B1CE
:105A300001EB410202EBC10200EB820202F8345F8B
:105A4000567082F80290D3700EE001EB410404EB33
:105A5000C10400EB8404926904F8342F170A6770BC
:105A6000170CA770120EE270491CC9B204297FF608
:105A700093AE0120BDE8F083A03E00202DE9FE4F4B
:105A80000446D9480290DC480190DC480090002090
:105A90000226DFF85093DFF854B3D54ADFF854A359
:105AA000014607460546731E10E000BF0AEB400C96
:105AB000401C9CF82480C0B241449CF814809CF89F
:105AC00034C047446544C9B2FFB2EDB29842EDDB41
:105AD0000020034604EB000C401CC0B28CF81030D0
:105AE0000428F7D306EBC60000EB461C0BEB4C0C6E
:105AF0009CF8020004F8140F00206070A070E070A1
:105B00009CF840302371607106EB8603A07103EBB3
:105B1000861CE07112F81C3023726072A07202EBD6
:105B20004C03E07293F8288084F80C806073A073B3
:105B3000E07312F81C2022746074A074E07493F86F
:105B4000282022756075A075E07501EBC10000EB9F
:105B500041120BEB42009A46B0F89E004FF003084A
:105B6000143C10B184F82C8005E0491CC8B2FCF745
:105B700021FA84F82C0007EB071000EB4001009895
:105B800000EB4100B0F8C41011B184F8308003E09C
:105B900090F8BE1084F83010C5EBC50101EB81020E
:105BA000019901EB4201B1F880201AB1414684F815
:105BB000348004E011F87A2F84F83420897884F84E
:105BC0003810B0F8C41011B184F83C8003E090F8AC
:105BD000C00084F83C00002504F82D5F6570A570B6
:105BE00025716571A57125726572A572257365733E
:105BF000A57325746574A5749AF82800E07425755A
:105C00006575A5759AF82800E07525766576A57600
:105C100000202D3C2118401CC0B281F8485020289B
:105C2000F8D3029806EB860100EBC107F88B40B170
:105C300084F8685084F8695084F86A5084F86B508E
:105C40000BE0786884F86800010A84F86910010C98
:105C500084F86A10000E84F86B00F88BDFF8A081DE
:105C600040B184F86C5084F86D5084F86E5084F81C
:105C70006F5013E009EBC610B0F92A00FAF7CFFB1A
:105C80004146FAF75CFB84F86C00010A84F86D1059
:105C9000010C84F86E10000E84F86F00F88B40B190
:105CA00084F8705084F8715084F8725084F87350FE
:105CB00013E009EBC610B0F90200FAF7B0FB414659
:105CC000FAF73DFB84F87000010A84F87110010CAA
:105CD00084F87210000E84F87300F88B40B184F8D9
:105CE000745084F8755084F8765084F8775013E037
:105CF00009EBC610B0F92A00FAF791FB4146FAF712
:105D00001EFB84F87400010A84F87510010C84F8F5
:105D10007610000E84F87700F88B40B184F8785044
:105D200084F8795084F87A5084F87B5013E009EBBA
:105D3000C610B0F95200FAF772FB4146FAF7FFFAC3
:105D400084F87800010A84F87910010C84F87A103C
:105D5000000E84F87B00F88B58B1762084F87C0024
:105D60007F2084F87D00FF2084F87E0084F87F5037
:105D70000BE0B86984F87C00010A84F87D10010CFE
:105D800084F87E10000E84F87F00F88B84F8805031
:105D900084F8815084F8825084F88350F88B84F81A
:105DA000845084F8855084F8865084F88750F88BA6
:105DB00084F8885084F8895084F88A5084F88B508D
:105DC000F88B84F88C5084F88D5084F88E5084F8C9
:105DD0008F50F88B04F8905F01206570A570E57016
:105DE000BDE8FE8FA4410020A03E0020A449002071
:105DF000C44E0020A8360020483200203E38002043
:105E0000CDCCCC3DF0B503259C4C9D4E9D4B002246
:105E100011468718521CD2B23974042AF9D305EB03
:105E2000C50202EB451206EB4202967800F8146FA9
:105E300041708170C17092F840200271417105EB90
:105E40008502817102EB8516C17113F8162002726A
:105E50004172817203EB4602C17212F8287F077308
:105E600041738173C17313F81670077441748174A0
:105E7000C1741778077541758175C17513F816706F
:105E8000077641768176C1761778077741778177F3
:105E9000C17713F8163080F8203080F8211080F890
:105EA000221080F82310137880F8243080F8251011
:105EB00080F8261080F82710137880F8283080F8B2
:105EC000291080F82A1080F82B10137880F82C30D5
:105ED00080F82D1080F82E1080F82F10127880F89E
:105EE000302080F8311080F8321080F83310002212
:105EF00014388318521CD2B283F84810202AF8D3E1
:105F000005EB850304EBC302D58B45B180F868101F
:105F100080F8691080F86A1080F86B100CE054F873
:105F2000333080F868301C0A80F869401C0C80F817
:105F30006A401B0E80F86B30D38B43B180F86C1035
:105F400080F86D1080F86E1080F86F100BE0936889
:105F500080F86C301C0A80F86D401C0C80F86E4094
:105F60001B0E80F86F30D38B43B180F8701080F82F
:105F7000711080F8721080F873100BE0D36880F80D
:105F800070301C0A80F871401C0C80F872401B0EA7
:105F900080F87330D38B43B180F8741080F875109B
:105FA00080F8761080F877100BE0136980F8743071
:105FB0001C0A80F875401C0C80F876401B0E80F897
:105FC0007730D38B43B180F8781080F8791080F85F
:105FD0007A1080F87B100BE0536980F878301C0A47
:105FE00080F879401C0C80F87A401B0E80F87B30DA
:105FF000D38B5BB1762380F87C307F2380F87D30B3
:10600000FF2380F87E3080F87F100BE0936980F8E2
:106010007C301C0A80F87D401C0C80F87E401B0EF2
:1060200080F87F30D38B80F8801080F8811080F862
:10603000821080F88310D38B80F8841080F885104C
:1060400080F8861080F88710D38B80F8881080F84D
:10605000891080F88A1080F88B10D38B80F88C1010
:1060600080F88D1080F88E1080F88F10D28B00F899
:10607000901F41708170C1700120F0BDA03E0020D2
:10608000A4490020C44E0020F0B504259C4C9D4E30
:106090009D4B002211468718521CD2B23974042A33
:1060A000F9D305EBC50202EB451206EB42029678E6
:1060B00000F8146F41708170C17092F84020027135
:1060C000417105EB8502817102EB8516C17113F8F0
:1060D000162002724172817203EB4602C17212F8FD
:1060E000287F077341738173C17313F816700774A7
:1060F00041748174C1741778077541758175C175D4
:1061000013F81670077641768176C176177807778F
:1061100041778177C17713F8163080F8203080F806
:10612000211080F8221080F82310137880F8243092
:1061300080F8251080F8261080F82710137880F852
:10614000283080F8291080F82A1080F82B10137856
:1061500080F82C3080F82D1080F82E1080F82F1049
:10616000127880F8302080F8311080F8321080F8F2
:106170003310002214388318521CD2B283F848100E
:10618000202AF8D305EB850304EBC302D58B45B178
:1061900080F8681080F8691080F86A1080F86B1039
:1061A0000CE054F8333080F868301C0A80F86940FD
:1061B0001C0C80F86A401B0E80F86B30D38B43B107
:1061C00080F86C1080F86D1080F86E1080F86F10F9
:1061D0000BE0936880F86C301C0A80F86D401C0C52
:1061E00080F86E401B0E80F86F30D38B43B180F87F
:1061F000701080F8711080F8721080F873100BE046
:10620000D36880F870301C0A80F871401C0C80F84C
:1062100072401B0E80F87330D38B43B180F874103A
:1062200080F8751080F8761080F877100BE013690D
:1062300080F874301C0A80F875401C0C80F8764099
:106240001B0E80F87730D38B43B180F8781080F83C
:10625000791080F87A1080F87B100BE0536980F891
:1062600078301C0A80F879401C0C80F87A401B0EAC
:1062700080F87B30D38B5BB1762380F87C307F2332
:1062800080F87D30FF2380F87E3080F87F100BE0AF
:10629000936980F87C301C0A80F87D401C0C80F8E3
:1062A0007E401B0E80F87F30D38B80F8801080F802
:1062B000811080F8821080F88310D38B80F88410CE
:1062C00080F8851080F8861080F88710D38B80F8CE
:1062D000881080F8891080F88A1080F88B10D38B92
:1062E00080F88C1080F88D1080F88E1080F88F1058
:1062F000D28B00F8901F41708170C1700120F0BDF9
:10630000A03E0020A4490020C44E0020F0B5052581
:106310009C4C9D4E9D4B002211468718521CD2B2B8
:106320003974042AF9D305EBC50202EB451206EBDA
:106330004202967800F8146F41708170C17092F833
:1063400040200271417105EB8502817102EB8516D7
:10635000C17113F8162002724172817203EB46027A
:10636000C17212F8287F077341738173C17313F8E8
:106370001670077441748174C1741778077541757C
:106380008175C17513F81670077641768176C176EE
:106390001778077741778177C17713F8163080F83F
:1063A000203080F8211080F8221080F82310137814
:1063B00080F8243080F8251080F8261080F8271007
:1063C000137880F8283080F8291080F82A1080F897
:1063D0002B10137880F82C3080F82D1080F82E10B8
:1063E00080F82F10127880F8302080F8311080F873
:1063F000321080F83310002214388318521CD2B2A5
:1064000083F84810202AF8D305EB850304EBC30278
:10641000D58B45B180F8681080F8691080F86A1053
:1064200080F86B100CE054F8333080F868301C0AA8
:1064300080F869401C0C80F86A401B0E80F86B30B5
:10644000D38B43B180F86C1080F86D1080F86E101B
:1064500080F86F100BE0936880F86C301C0A80F8AD
:106460006D401C0C80F86E401B0E80F86F30D38B93
:1064700043B180F8701080F8711080F8721080F8C5
:1064800073100BE0D36880F870301C0A80F87140FC
:106490001C0C80F872401B0E80F87330D38B43B114
:1064A00080F8741080F8751080F8761080F87710F6
:1064B0000BE0136980F874301C0A80F875401C0CDE
:1064C00080F876401B0E80F87730D38B43B180F88C
:1064D000781080F8791080F87A1080F87B100BE043
:1064E000536980F878301C0A80F879401C0C80F8D9
:1064F0007A401B0E80F87B30D38B5BB1762380F81B
:106500007C307F2380F87D30FF2380F87E3080F858
:106510007F100BE0936980F87C301C0A80F87D4086
:106520001C0C80F87E401B0E80F87F30D38B80F8E7
:10653000801080F8811080F8821080F88310D38B4F
:1065400080F8841080F8851080F8861080F8871015
:10655000D38B80F8881080F8891080F88A1080F832
:106560008B10D38B80F88C1080F88D1080F88E10F3
:1065700080F88F10D28B00F8901F41708170C1702D
:106580000120F0BDA03E0020A4490020C44E002000
:10659000F0B506259C4C9D4E9D4B00221146871858
:1065A000521CD2B23974042AF9D305EBC50202EBAE
:1065B000451206EB4202967800F8146F4170817024
:1065C000C17092F840200271417105EB8502817122
:1065D00002EB8516C17113F81620027241728172A6
:1065E00003EB4602C17212F8287F0773417381736F
:1065F000C17313F81670077441748174C1741778ED
:10660000077541758175C17513F816700776417667
:106610008176C1761778077741778177C17713F84C
:10662000163080F8203080F8211080F8221080F891
:106630002310137880F8243080F8251080F8261075
:1066400080F82710137880F8283080F8291080F817
:106650002A1080F82B10137880F82C3080F82D1039
:1066600080F82E1080F82F10127880F8302080F8F3
:10667000311080F8321080F833100022143883185B
:10668000521CD2B283F84810202AF8D305EB8503B8
:1066900004EBC302D58B45B180F8681080F869100F
:1066A00080F86A1080F86B100CE054F8333080F8F2
:1066B00068301C0A80F869401C0C80F86A401B0E88
:1066C00080F86B30D38B43B180F86C1080F86D107C
:1066D00080F86E1080F86F100BE0936880F86C30D3
:1066E0001C0A80F86D401C0C80F86E401B0E80F870
:1066F0006F30D38B43B180F8701080F8711080F840
:10670000721080F873100BE0D36880F870301C0AA8
:1067100080F871401C0C80F872401B0E80F87330BA
:10672000D38B43B180F8741080F8751080F8761020
:1067300080F877100BE0136980F874301C0A80F839
:1067400075401C0C80F876401B0E80F87730D38B98
:1067500043B180F8781080F8791080F87A1080F8CA
:106760007B100BE0536980F878301C0A80F8794080
:106770001C0C80F87A401B0E80F87B30D38B5BB109
:10678000762380F87C307F2380F87D30FF2380F8EB
:106790007E3080F87F100BE0936980F87C301C0A13
:1067A00080F87D401C0C80F87E401B0E80F87F3006
:1067B000D38B80F8801080F8811080F8821080F8E8
:1067C0008310D38B80F8841080F8851080F88610B1
:1067D00080F88710D38B80F8881080F8891080F8B3
:1067E0008A1080F88B10D38B80F88C1080F88D1075
:1067F00080F88E1080F88F10D28B00F8901F4170B7
:106800008170C1700120F0BDA03E0020A44900208D
:10681000C44E0020F0B507259C4C9D4E9D4B002298
:1068200011468718521CD2B23974042AF9D305EBE9
:10683000C50202EB451206EB4202967800F8146F8F
:1068400041708170C17092F840200271417105EB76
:106850008502817102EB8516C17113F81620027250
:106860004172817203EB4602C17212F8287F0773EE
:1068700041738173C17313F8167007744174817486
:10688000C1741778077541758175C17513F8167055
:10689000077641768176C1761778077741778177D9
:1068A000C17713F8163080F8203080F8211080F876
:1068B000221080F82310137880F8243080F82510F7
:1068C00080F8261080F82710137880F8283080F898
:1068D000291080F82A1080F82B10137880F82C30BB
:1068E00080F82D1080F82E1080F82F10127880F884
:1068F000302080F8311080F8321080F833100022F8
:1069000014388318521CD2B283F84810202AF8D3C6
:1069100005EB850304EBC302D58B45B180F8681005
:1069200080F8691080F86A1080F86B100CE054F859
:10693000333080F868301C0A80F869401C0C80F8FD
:106940006A401B0E80F86B30D38B43B180F86C101B
:1069500080F86D1080F86E1080F86F100BE093686F
:1069600080F86C301C0A80F86D401C0C80F86E407A
:106970001B0E80F86F30D38B43B180F8701080F815
:10698000711080F8721080F873100BE0D36880F8F3
:1069900070301C0A80F871401C0C80F872401B0E8D
:1069A00080F87330D38B43B180F8741080F8751081
:1069B00080F8761080F877100BE0136980F8743057
:1069C0001C0A80F875401C0C80F876401B0E80F87D
:1069D0007730D38B43B180F8781080F8791080F845
:1069E0007A1080F87B100BE0536980F878301C0A2D
:1069F00080F879401C0C80F87A401B0E80F87B30C0
:106A0000D38B5BB1762380F87C307F2380F87D3098
:106A1000FF2380F87E3080F87F100BE0936980F8C8
:106A20007C301C0A80F87D401C0C80F87E401B0ED8
:106A300080F87F30D38B80F8801080F8811080F848
:106A4000821080F88310D38B80F8841080F8851032
:106A500080F8861080F88710D38B80F8881080F833
:106A6000891080F88A1080F88B10D38B80F88C10F6
:106A700080F88D1080F88E1080F88F10D28B00F87F
:106A8000901F41708170C1700120F0BDA03E0020B8
:106A9000A4490020C44E0020F0B508259C4C9D4E12
:106AA0009D4B002211468718521CD2B23974042A19
:106AB000F9D305EBC50202EB451206EB42029678CC
:106AC00000F8146F41708170C17092F8402002711B
:106AD000417105EB8502817102EB8516C17113F8D6
:106AE000162002724172817203EB4602C17212F8E3
:106AF000287F077341738173C17313F8167007748D
:106B000041748174C1741778077541758175C175B9
:106B100013F81670077641768176C1761778077775
:106B200041778177C17713F8163080F8203080F8EC
:106B3000211080F8221080F82310137880F8243078
:106B400080F8251080F8261080F82710137880F838
:106B5000283080F8291080F82A1080F82B1013783C
:106B600080F82C3080F82D1080F82E1080F82F102F
:106B7000127880F8302080F8311080F8321080F8D8
:106B80003310002214388318521CD2B283F84810F4
:106B9000202AF8D305EB850304EBC302D58B45B15E
:106BA00080F8681080F8691080F86A1080F86B101F
:106BB0000CE054F8333080F868301C0A80F86940E3
:106BC0001C0C80F86A401B0E80F86B30D38B43B1ED
:106BD00080F86C1080F86D1080F86E1080F86F10DF
:106BE0000BE0936880F86C301C0A80F86D401C0C38
:106BF00080F86E401B0E80F86F30D38B43B180F865
:106C0000701080F8711080F8721080F873100BE02B
:106C1000D36880F870301C0A80F871401C0C80F832
:106C200072401B0E80F87330D38B43B180F8741020
:106C300080F8751080F8761080F877100BE01369F3
:106C400080F874301C0A80F875401C0C80F876407F
:106C50001B0E80F87730D38B43B180F8781080F822
:106C6000791080F87A1080F87B100BE0536980F877
:106C700078301C0A80F879401C0C80F87A401B0E92
:106C800080F87B30D38B5BB1762380F87C307F2318
:106C900080F87D30FF2380F87E3080F87F100BE095
:106CA000936980F87C301C0A80F87D401C0C80F8C9
:106CB0007E401B0E80F87F30D38B80F8801080F8E8
:106CC000811080F8821080F88310D38B80F88410B4
:106CD00080F8851080F8861080F88710D38B80F8B4
:106CE000881080F8891080F88A1080F88B10D38B78
:106CF00080F88C1080F88D1080F88E1080F88F103E
:106D0000D28B00F8901F41708170C1700120F0BDDE
:106D1000A03E0020A4490020C44E00202DE9F04FE1
:106D20008FB00446C3480990C3480090C4480890F7
:106D3000C24BC64807904FF000099A7F0192DFF8D6
:106D400004B3DFF804A3521E4D464E464F46484654
:106D5000082A1AD300200FB0BDE8F08F009901EB8C
:106D60004001401C91F82480C0B208EB090C0CF0E3
:106D7000FF0991F814C0654491F834C091F84410AB
:106D800066443944EDB2F6B2CFB29042E6DB282039
:106D900009EBC901E07201EB4911987F0AEB410A46
:106DA0006074BAF89E004FF0030810B184F81280A6
:106DB00005E009F10100C0B2FBF7FCF8A07405EB97
:106DC000051000EB40010BEB4105B5F8C40010B114
:106DD00084F8138002E095F8BE00E074FBF7B6FE7D
:106DE0009B490860C6EBC60000EB8001089800EBE9
:106DF0004106B6F8800018B1404684F8148004E0DB
:106E000096F87A00207596F87C006075B5F8C40095
:106E100010B184F8168002E095F8C000A07507EB69
:106E2000870000EB8711099800EB4100B0F80E11C4
:106E300011B184F8178002E090F80801E075079816
:106E40004FF0A50B90F8F2002076BAF89E009AF861
:106E50007400607684F81AB084F81BB0DDE9000194
:106E600000EB4107788C01280CD9BAF8F00010B17A
:106E700084F81C8008E009F10200C0B2FBF79AF820
:106E8000207701E084F81CB0788A012815D9B5F87C
:106E90002A0110B14046607704E095F8240160773C
:106EA00095F8260184F82000788E012820D9B6F8BC
:106EB000C60020B14046A07706E05846EBE796F8BA
:106EC000C000A07796F8C200E07784F821B084F87B
:106ED00022B084F823B084F824B084F825B0788CEC
:106EE00002280FD9BAF8420120B184F826800BE0BD
:106EF0005846E0E709F10300C0B2FBF75BF884F8FD
:106F0000260001E084F826B0788A022819D9B5F85D
:106F1000900120B14FEA080084F8270005E095F8B9
:106F20008A0184F8270095F88C0184F82A00788E6D
:106F3000022823D9B6F80C0128B1404684F828006D
:106F400007E05846E8E796F8060184F8280096F826
:106F5000080184F8290084F82BB084F82CB084F858
:106F60002DB084F82EB084F82FB0788C03280FD978
:106F7000BAF8940120B184F830800BE05846DDE780
:106F800009F10400C0B2FBF715F884F8300001E005
:106F900084F830B0788A032819D9B5F8F60118B109
:106FA00084F8318084F8348095F8F00184F8310059
:106FB00095F8F20184F83400788E042838D9B6F8B0
:106FC000520140B14FEA080084F8320009E0584607
:106FD00084F831B0EEE796F84C0184F8320096F868
:106FE0004E0184F8330084F835B084F836B084F864
:106FF00037B0174884F838B084F839B00068B0F575
:10700000005F13D2002004F8140F6070A070E070CD
:10701000A072E0722073607320756075A075E075D2
:10702000A077E07784F8200084F82100012092E620
:107030005846C9E7C44E0020A8360020A4370020D7
:10704000483200203E380020A44900206457002028
:10705000240300202DE9F041654904466148897FF9
:10706000614DDFF888C1A1F1510E002247277F262C
:10707000FF23BEF10E0F24D2607C00EB80000CEBEE
:10708000C005A5F58055B5F89E0320B1A774E67438
:1070900023756275A3E0D5F8800305F56075F9F7EF
:1070A000CCF9000EA0742868F9F7C7F9000CE07459
:1070B0002868F9F7C2F9000A20752868F9F7BDF9C0
:1070C00086E0A1F1610CBCF10E0F3ED2607C05EBB5
:1070D000C010A0F54050B0F87A1059B1A774E6740A
:1070E00023756275A775E67523766276A776E676D0
:1070F00023776277B0F90010090EA174B0F900107F
:10710000090CE1740188090A217501786175B0F9EB
:107110002810090EA175B0F92810090CE175018D30
:10712000090A217690F828106176B0F95010090EFE
:10713000A176B0F95010090CE176B0F85010090AA8
:10714000217790F85000607749E0A1F171050E2D8C
:1071500045D3103D0E2D42D3603D022D3AD2B0F8FA
:107160007A1061B1A774E67423756275A775E67528
:1071700023766276A776E676237762772FE0B0F9FA
:107180000010090EA174B0F90010090CE174018817
:10719000090A217501786175B0F92810090EA174EA
:1071A000B0F92810090CE174018D090A217590F8D5
:1071B00028106175B0F95010090EA174B0F9501083
:1071C000090CE174B0F85010090A217590F85000CC
:1071D000607504E0E42902D00020BDE8F0810120C0
:1071E000FBE7000020410020A4410020A03E002039
:1071F000A437002010B50C4A002100BF52F82130FE
:107200001C0E00EB81031C7452F82140240C5C74AA
:1072100032F82140240A9C7412F82140491CDC7485
:107220000829EBDB012010BD2C0300202DE9F041E3
:107230001B4E04460025B6F90000F9F7F0F8194F87
:107240003946F9F77CF82074010A6174010CA174C5
:10725000000EE074B6F92800F9F7E1F83946F9F7BD
:107260006EF82075010A6175010CA175000EE075BC
:10727000B6F95000F9F7D3F83946F9F760F82076F7
:10728000010A6176010CA176000EE076A520611955
:107290006D1CEDB20877E42DF9D30120BDE8F08133
:1072A000204100200000B43B72B6012080F3138817
:1072B000BFF34F8F05480168054A01F4E0611143AF
:1072C0000160BFF34F8F00BFFDE700000CED00E051
:1072D0000400FA0510B5002306E000BF30F8024BA9
:1072E00021F813405B1C9BB29342F7D310BD000002
:1072F0002DE9F05FA0F1006415468A468346B4F597
:10730000002F5FD2FBF700FBE70AC4F34906C6F57E
:107310008064A54200D82C46DFF8AC904FF00060A6
:1073200000EBC72080464FF480622749FFF7D2FF69
:1073300000204FF6FF7106E0331839F813208A4217
:1073400003D1401C80B2A042F6D3A0422ED24046C8
:10735000F9F7BCFF4CF25030FAF706F81B48016908
:1073600021F0020101610020494606E03AF81020B0
:107370008319401C21F8132080B2A042F6D3124991
:1073800040464FF4806200BF00F022F8A54215D0BD
:10739000281B0AEB440A0BEB440B002685B24FF482
:1073A00080647F1CA542B9D82C46B7E74CF2503018
:1073B000F9F7DAFF224651465846E5E7BDE8F05FA7
:1073C000FBF758BABDE8F09F426800200020024059
:1073D0002DE9F04116460F46054600240AE000BF9D
:1073E00037F81420002329460120FBF74DFA641CCE
:1073F000A4B2AD1CB442F3D3BDE8F0812DE9FF5F28
:10740000054659480390594802900020834681461A
:1074100080460090AA20287000206870A121A970E1
:107420001121DFF840A1E97085F804004FEA4860B7
:10743000010E00206C180AEB48076071A07129E06A
:1074400000EB0901C1EBC10101EB8102039901EBE2
:107450004201B1F880201AB1627942F0100205E0D1
:10746000B1F87A201AB1627942F001026271BAF879
:107470000A206AB1B1F884201AB1617941F0200183
:1074800005E0B1F87C1019B1617941F00201617138
:10749000401CC0B2B98E8142D2D8484400F0FF09E6
:1074A000002021E000EB0B0101EB011101EB410297
:1074B000029901EB4201B1F8C4203AB1617941F07F
:1074C00080016171A17941F055010AE0B1F8BE2057
:1074D0001AB1627942F008026271B1F8C01009B1C4
:1074E0000121A171401CC0B2B98A8142DAD8584446
:1074F00000F0FF0B002612E03044401C0190C0B2A7
:10750000FAF758FD012828D00198C0B2FAF752FDC9
:1075100018B1607900F040006071761CF6B2B88C4A
:10752000B0420098E8D83044C0B2009008F10100A1
:1075300000F0FF08B8F1080FFFF478AF0C480068BE
:10754000B0F5005F07D2002001462A18401CC0B2E7
:1075500051711028F9D3BDE8FF9F607940F0040015
:10756000DAE70000A8360020483200203E3800202C
:10757000240300202DE9F04186B00546194F1A4E2C
:107580001A4C14216846F8F770FEB4F81D00DFF8B5
:10759000608040BAADF80000207D062804D10122A9
:1075A00041466846F9F718FF012241466846F9F757
:1075B00005FFBDF80000A7F84000A6F86000000A2B
:1075C0002874BDF80010C9B26974627F904206D178
:1075D000A07F814203D1012006B0BDE8F0810020E8
:1075E000FAE70000483200203E380020A43700208F
:1075F00064F00708094908B5074848624BF6BB30F4
:10760000ADF8020045F25550ADF8000002220449E1
:107610006846F9F7E1FE08BDBBBB5555CC09002013
:107620007AF00708094808B54FF0AA314162080C02
:10763000ADF80000ADF80200022205496846F9F7EE
:10764000CBFE012080F3138802F0B6F8CC090020AD
:107650007AF00708012002F07BFDFBE78CB00024E4
:10766000FE48DFF8FCB3A14626460A90FD48089084
:10767000FE480090FE48FC4D27460481A4462A8817
:107680000BE000BF05EB4103491CB3F814809B8C51
:1076900046443B44B6B29FB2018101898A42F1D887
:1076A000E046A0F808C082460A2002F051FD4FF4DF
:1076B0008061F048FBF73DFA9AF80000B0B100266F
:1076C000AAF80880374650462A880AE005EB4103AD
:1076D000491CB3F814C09B8C66443B44B6B29FB2BD
:1076E000018101898A42F1D88AF80080BBF8020042
:1076F00030B1B9F1030F7DD0B9F1060F7BD038E17D
:1077000044B1032C4BD0062C76D0092C75D00C2C10
:1077100074D005E1288AE8B3A88802283ED0062163
:10772000D548FCF74DFBD449020A8A71C871002282
:107730004FF48051D148FBF704FA502002F004FACC
:107740000822CD49CE48FCF7F0F902E0012002F012
:10775000FFFCCB4890F839002128F7D00122110313
:10776000C648FBF7EEF9C44A107800EB001000EBB6
:107770004001089800EB4100A0F58050B0F8041AD1
:10778000491CA0F8041A1078A0F11001B14202DAE5
:10779000401C01E002E011201070C1E00324B5F8A4
:1077A0006C0060B3B44806211830FCF709FBB249FD
:1077B000020A18318A71C87100224FF48051AF4813
:1077C000FBF7BFF9502002F0BFF9AB496423082250
:1077D0001831AB48FCF750F9502002F0B5F90122FE
:1077E0001103A648FBF7ADF90098B0F87E003C28DD
:1077F0000ED905E09BE0B8E010E02AE06BE00CE079
:1078000000993C20A1F87E000099A1F8780087E05B
:107810000099401CA1F87E0082E00624E889B8B1F6
:10782000954806212030FCF7CBFA9349020A203113
:107830008A71C87100224FF480519048FBF781F99A
:10784000502002F081F98C496423082220315CE049
:107850000924688AD0B3E888C0B30E218948FCF7B0
:10786000AFFA8849020A8A73C87300224FF4805124
:107870008248FBF766F9502002F066F96423102273
:1078800080497F48FCF7F8F8502002F05DF90122AA
:1078900011037A48FBF755F97A48007800EBC001EC
:1078A00001EB40110A9800EB4101A1F58051B1F8BC
:1078B0001006322802D8401CA1F810067149087839
:1078C000A0F12102BA4202DA401C01E002E02120CC
:1078D000087025E00C24B5F86E0030B36648062128
:1078E0001030FCF76DFA6449020A10318A71C871D0
:1078F00000224FF480516148FBF723F9502002F039
:1079000023F95D496423082210315D48FCF7B4F87F
:10791000502002F019F9012211035848FBF711F920
:1079200059480068012837D02BE00024BCE600222B
:107930004FF480515148FBF704F9502002F004F94C
:107940005248534902884E48FCF7EFF802E0012004
:1079500002F0FEFB4A4890F839002128F7D00122B6
:1079600011034648FBF7EDF803E0ABF802804FF057
:10797000000909F1010000F0FF09434800680128EF
:1079800002D0022C69D0E2E0B9F1030F04D9ABF8C0
:1079900002804FF0000987E63B483E4AC0F800806D
:1079A0001078A0F110010F297ED85079010290794A
:1079B000084301905078032805D0062803D0012100
:1079C000AAF80C10C1E033488078022803D00120C7
:1079D000AAF80C00B9E005212E48FCF7F1F901994D
:1079E0008842F4D1BAF80C00B0BB2A490A7802EBFD
:1079F000021202EB4203089A02EB4302A2F5805204
:107A0000A2F8FC890A7802EB021202EB4203089A00
:107A100002EB4302A2F58052A2F8FE8948780328BF
:107A200040D10878CA7800EB001000EB40030898BA
:107A300000EB4300A0F58050A0F8A02908780A794F
:107A400000EB001000EB4003089800EB4300A0F5AA
:107A50008050A0F8C82920E068E080E0A449002018
:107A6000A43700203E380020A83600202041002006
:107A7000080000200010014020010020000C0140FF
:107A8000AC2A0020EC02002010030020C4090020D2
:107A90005E3700200028002006E00878103880B209
:107AA00001F014FE0324FFE5A0F170010F293ED878
:107AB00000980123A0F87E305078032805D00628CE
:107AC00003D000BFAAF80C303FE091780829F9D222
:107AD0003648C91CFCF774F9BAF80C10504629BB9B
:107AE00032494A78032A30D1B0F80AC0BCF1140FE9
:107AF00016D2009BA3F8788031F8032F009B52BA6E
:107B000023F81C204A8853BA009A02EB4C020CF16D
:107B1000010C1385898849BAA2F85010A0F80AC050
:107B20001FFA8CF1142910D1AAF80A800DE0A0F1F7
:107B300020010F2902D8FAF7BBFA06E0E4280BD09F
:107B400081380E2801D8FAF7F5F9AAF80C800F2C25
:107B500026D2641CE4B224E0FAF766FAF5E714488A
:107B60000078112819D01138AAF80800BAF80800CE
:107B700000EB001000EB4001089800EB4100B0F86A
:107B80005C10491C89B2A0F85C100329E1D90B21D3
:107B900020F85C1F01214180DBE7AAF80860E5E7D7
:107BA0000024282002F0D4FA7EE5000000280020FE
:107BB000200100208EB0FD480C90FE480790FF4841
:107BC000FD4D0990FE4800270290B5F86600DFF8E9
:107BD000E0933E46BB46022802D10320A5F866008A
:107BE000F84C0022E281298809E000BF05EB400340
:107BF000761C9B8E401C3B449FB2B6B2E081E0896C
:107C00008142F3D8B5F8660010F0FF0F16D0C0B26D
:107C100070431FFA80F89246E2810A2002F098FA37
:107C20004FF48061E848FAF784FF207830B30027EA
:107C3000B5F866003E46022802D004E0B046EAE706
:107C40000320A5F86600A4F80EA05346298808E092
:107C500005EB4002761C928E401C3A4497B2B6B2B5
:107C6000E081E0898142F3D8B5F8660010F0FF0F9B
:107C70000BD0C0B270431FFA80F82370B9F800002F
:107C800028B1A07803287BD0EFE1B046F5E7607813
:107C9000002871D1A889002874D02889022871D0C1
:107CA000C8B1CA480178C1EBC10101EB8102079953
:107CB00001EB4201A1F58051B1F82423521CA1F837
:107CC000242301783039B9422DDAE178491CE1707A
:107CD000303101702BE0BD490878012809D001201E
:107CE000087007980799B0F84400401CA1F84400B8
:107CF0001DE0E078B84202D3504684F803A0C0B239
:107D0000401CC0B20122E07002EB40020A70C0EBDE
:107D1000C00000EB8001079800EB410131F8440FEF
:107D2000401C088003E0312101700120E070062131
:107D3000A648FCF745F8A5496082020A8A71C87115
:107D400000224FF40051A248FAF7FBFE502001F048
:107D5000FBFE08229D499F48FBF7E7FE02E0012059
:107D600002F0F6F99B4890F839002128F7D001225B
:107D700051039748FAF7E5FE6078032804D069E0DC
:107D800056E1FFE7032060706889012802D00620D1
:107D9000607062E006219048FCF712F88E4960821C
:107DA000020A8A71C87100224FF400518848FAF71C
:107DB000C8FE502001F0C8FE2889012806D181495B
:107DC0000A230222491D8348FBF756FE642308223A
:107DD00081498048FBF750FE2889012806D179495E
:107DE0000A230222491D7B48FBF746FE502001F082
:107DF000ABFE012251037648FAF7A3FE76480178DC
:107E0000C1EBC10101EB8102079901EB4201A1F530
:107E10000051B1F8C42E3C2A0FD93C22A1F8C42E3F
:107E20000178C1EBC10101EB8103079901EB43012B
:107E3000A1F50051A1F8BC2E02E0521CA1F8C42EFD
:107E400001787A1EA1F14103934201DA491C00E056
:107E5000412101706078062848D1B5F8640018B156
:107E6000012804D0022845D00920607080E05748DE
:107E700006212830FBF7A4FF544960822831020A0A
:107E80008A71C87100224FF400515148FAF759FE27
:107E9000502001F059FE4D49082228314D48FBF78A
:107EA00044FE02E0012002F053F94A4890F83900FC
:107EB0002128F7D0012251034548FAF742FE4349F1
:107EC0002831087800EB8002099800EBC200A0F589
:107ED0008050B0F8A223521CA0F8A2230878A0F189
:107EE000510241E0401C00E05120087060780928F0
:107EF0003ED095E0354806212030FBF761FF33493D
:107F000060822031020A8A71C87100224FF4005148
:107F10002F48FAF716FE502001F016FE2B490822D2
:107F200020312C48FBF701FE02E0012002F010F99D
:107F3000284890F839002128F7D00122510324481D
:107F4000FAF7FFFD21492031087800EB80020998FB
:107F500000EBC200A0F58050B0F8A223521CA0F89C
:107F6000A2230878A0F15002731E9A42BCDAB9E746
:107F7000B5F8660090B3154806213030FBF720FFB6
:107F8000124960823031020A8A71C87100224FF4AE
:107F900000510F48FAF7D5FD502001F0D5FD0B49EF
:107FA000082230310B48FBF7C0FD1BE0C82D002034
:107FB000A437002048320020A8360020A03E002030
:107FC000A4410020080000200010014028010020EA
:107FD000000C01402C2A0020FC02002025E001209A
:107FE00002F0B6F8FE4890F839002128F7D00122B7
:107FF0005103FC48FAF7A5FDFB4902980A7800EB0B
:10800000C210A0F53C5082380288521C02800878C9
:10801000A0F16002424501DA401C00E061200870D6
:10802000F2480068012835D027E084F801A0F4E583
:1080300000224FF40051EB48FAF783FD502001F085
:1080400083FDEB48EB490288E548FBF76EFD02E053
:10805000012002F07DF8E24890F839002128F7D09D
:1080600001225103DF48FAF76CFDA078DF49401C7C
:10807000C0B2A0700968012905D0607802287CD0C0
:1080800008287BD0EEE2032804D9A9F800A084F8E0
:1080900002A0C2E5D548C0F800A0D74884F804A0E3
:1080A00081784218D178127942EA0122628210F86E
:1080B0000B10A1F130020F2A02D94A1E0F2A7DD8D7
:1080C000CD4901EB0B0000904078032801D0062831
:1080D0000AD100988078042806D10721C648FBF70A
:1080E0006FFE618A884201D001202071009A0098B9
:1080F000C1495278B0F80300032AC3D12279002A7B
:10810000C0D111F80B20012A524614D0E378C3EBFA
:10811000C30303EB830C079B03EB4C031A87B6499D
:108120005A8711F80B10012909D0E178F8F742FAC3
:10813000288930B10BE0079B1A87079BEFE70021E6
:10814000F4E7AD48002110F80B00F8F7C9FAAA4887
:1081500010F80B0001283AD0E0780C9900EBC0022F
:1081600001EBC201079AB1F90610B2F842204B4266
:10817000934201DC91420DDD01E02CE252E2C0EBC2
:10818000C00101EB8102079901EB4202118E491CEB
:10819000118608E0C0EBC00202EB8203079A02EBF3
:1081A0004302A2F830A0C0EBC00000EB80010798AA
:1081B00000EB4100028EB0F8401000E009E08A4276
:1081C00003D301860121818601E0A0F834A00320B9
:1081D00073E0A1F140020F2A72D8C1EBC10101EB9B
:1081E00081030799012201EB4301A1F58051A1F818
:1081F0001CA310F80B10C1EBC10101EB810307991F
:1082000001EB4301A1F50051A1F8C42E00EB0B01D5
:1082100000914978032904D0062902D00120207159
:108220004AE000988078042806D107217248FBF7BD
:10823000C7FD618A884201D00120207100994978E8
:10824000032939D12179B9BB6B4810F80B1000987C
:10825000B0F8030040BAF8F7ADF9208A082826D212
:10826000654A009912F80B300979C3EBC30303EB9D
:10827000830C079B090203EB4C0303EB4003A3F5BC
:108280000053A3F8901E12F80B20C2EBC20202EBBF
:108290008203079A02EB4302009B02EB4002A2F525
:1082A0000052DB781943A2F8901E401C208280B255
:1082B000082801D1A4F810A006206070ADE4FFE703
:1082C0000178A1F150020F2A73D8B5F86420012A71
:1082D00002D0022A6ED0EFE001EB810309994648F3
:1082E00001EBC301A1F580510122A1F8A22302787C
:1082F00002EB8203099A02EBC302A2F58052A2F8B4
:108300009CA3407804280AD13B488078202806D1D5
:1083100023213948FBF754FD618A884201D00120AE
:108320002071354800EB0B014978042940D12179AF
:10833000F1BB324942790A7082794A70C2788A70F8
:108340000279CA7010F80B200B6802EB820C099AB4
:1083500002EBCC02A2F58052C2F88033427B0A7055
:10836000827B4A70C27A8A70027BCA7010F80B2036
:108370000B6802EB820C099A02EBCC02A2F5805248
:10838000C2F88833427C0A70827C4A70C27B8A7051
:10839000027CCA7010F80B200B6802EB820C099A61
:1083A00002EBCC02A2F58052C2F88833427D02E093
:1083B00082E083E038E00A70827D4A70C27C8A7075
:1083C000027DCA7010F80B200B6802EB820C099A30
:1083D00002EBCC02A2F58052C2F89033427E0FE04D
:1083E0002C2A0020000C0140580100200803002026
:1083F000C409002018370020FC0E002028000020AF
:108400000A70827E4A70C27D8A70027ECA7010F83D
:108410000B000A6800EB8001099800EBC100A0F591
:108420008050C0F8942347E001EB810309999448F8
:1084300001EBC301A1F580510122A1F8A22302782A
:1084400002EB8203099A02EBC302A2F58052A2F862
:108450009CA3407804280AD189488078042806D152
:1084600007218748FBF7ACFC618A884201D00120D4
:10847000207107218248FBF7A3FCA5F8680080481B
:1084800000EB0B014978042916D12179A1B97D4966
:1084900002790A70C2784A7082798A704279CA7009
:1084A00010F80B000A6800EB8001099800EBC1008E
:1084B000A0F58050C0F880230920FEE660390F291E
:1084C00072D87149029B012291F800C003EBCC13D2
:1084D000A3F54053A3F87E200B78029901EBC3115A
:1084E000A1F54051A1F878A04178032904D00629CC
:1084F00002D00120207198E5614880780228F8D1E7
:1085000005215F48FBF75CFC618A8842F1D15C4938
:1085100001EB0B0040780328EDD120790028EAD147
:10852000B5F8660001281BD00328E4D111F80B0030
:10853000613880B20322B0FBF2F302FB1303E08147
:108540008BB3012B3CD0022BD5D1B0FBF2F20298B9
:1085500000EBC212B1F8030040BAA2F8D20064E501
:10856000B1F8030011F80B3042BA029800EBC310C7
:10857000A0F540504280B1F8030011F80B3042BA28
:10858000029800EBC310A0F540504285B1F80300FB
:1085900011F80B20029940BA01EBC211A1F540512C
:1085A000A1F8520041E500E05CE0B0FBF2F2029875
:1085B00000EBC212B1F8030040BAA2F8820034E521
:1085C000B0FBF2F2029800EBC212B1F8030040BA1D
:1085D000A2F8AA0029E5288900282B48A0F130003C
:1085E000007816D031281BD03138E081E089079916
:1085F000C0EBC00000EB800001EB4000018F491C84
:1086000089B20187032930D90B21018701214187D4
:108610002BE0012801D0E078E7E7A4F80EA0E5E719
:10862000E781E3E7B5F86400012811D0022812D0F1
:10863000D8B1E089512813D05138E081E08900EBAE
:108640008001099800EBC101888B401C88830CE0F5
:108650000D48083801E00C4810380078E081E8E760
:10866000E681EBE760780C2803D26078401C6070EC
:1086700001E084F801A0282001F06AFDD7E40000A1
:10868000FC0E002028000020580100201FB500200B
:10869000F74CF84FDFF8E093DFF8E08300900390A9
:1086A0000190A4F5F27B06460290322001F050FDC5
:1086B0004FF48061F248FAF73CFAD8F8001001292B
:1086C000F3D1F048C8F800600088B0F5967F07D86D
:1086D00099F80010A52914D199F801005A2854D10D
:1086E000B9F8001099F8030049BA0A0499F8021081
:1086F00042EA01210143E448814202D1FCF7EEF94C
:10870000D3E799F8001048463A293ED141783329F9
:108710003BD18178392938D1C178302935D1DB492D
:108720000A68832A05D0DBF81C10491CCBF81C1002
:10873000BBE7002511E000BF09EB450A0AF1010083
:10874000FCF709F8CA498439294408750AF101007F
:10875000FCF701F8CE4948556D1CCC480068C01E96
:1087600000EBD070B5EB600FE6DBC84DC849286858
:10877000C01E00EBD0704210BF48F7F75DFD2868BF
:10878000C01E00EBD07040102860C048006805286B
:108790008BDB801E81B24D46B748FBF711FB287872
:1087A000392808D06878012805D8A878952802D8F3
:1087B000E878502802D96879012806D0F888401C4A
:1087C000F8800120CBF81C00D5E1E879032801D01E
:1087D0000628F3D1FE80CBF81C605946ABF8146034
:1087E000888A3B182A5C401C80B25A7388824028D1
:1087F000F6D38E82888A2A5C2254401C80B28882FA
:108800001028F7D3DBF81C00DA460028DCD1287AE0
:108810004FF6FF7101EA00207881697A0843788178
:10882000732873D031DC29286FD011DCA0F110003F
:1088300018286AD2DFE800F06769696B69696969BD
:1088400069696969696969696F6969696969697388
:10885000522879D00ADC4328E6D002DC402854D1E3
:1088600062E0502872D05128F9D182E07028DBD024
:1088700006DC5328D8D0542847D0552845D190E05D
:10888000712873D0722840D193E0B0F5BF7F6ED0CD
:1088900015DC7A286CD008DCA0F17400062834D2EC
:1088A000DFE800F093979B9FA3A77E2875D02CDC70
:1088B0007B2873D07C2872D07D2826D1A9E041F294
:1088C0009512811A90426BD015DC41F22112A0EB77
:1088D0000201904271D009DCB0F5C07F6ED0B0F5D6
:1088E000C87F6CD0B0F5087F0FD1AAE0722967D09D
:1088F00073290AD1B2E0072907D2DFE801F0E5CDFC
:10890000D1D5D9DDE100FEF7CFFCDDE059E06148CB
:10891000FEF774FDD8E02046FEF700FA02E020469C
:10892000FCF768FC0090CFE02046F7F7C3FF00900B
:108930005046AAF81460818A6A5C6254491C89B264
:1089400081824029F7D3BFE017E0FFE7204600F01F
:1089500007FE00905046AAF81460818A6A5C62544F
:10896000491C89B281824029F7D3ADE01DE058E06F
:1089700043E0204600F01CFED4E72046FCF702FC52
:1089800000905046AAF81460818A6A5C6254491CBF
:1089900089B281824029F7D396E03EE031E034E0AD
:1089A00061E02046FEF756FBBCE72046F8F772F878
:1089B000B8E72046FCF748FBB4E746E035E038E08E
:1089C00048E02046FEF7D6FDACE72046F8F788F8E9
:1089D00032E02046FCF772FB2EE0204600F012FE4B
:1089E0002AE02046FBF7F2F826E02046FBF77EFA65
:1089F00022E02046F7F71CFF1EE0204600F022FB95
:108A000090E72046FBF746F917E02046FBF7A4F96C
:108A100013E02046FBF76EF90FE02046FBF7A6F8BF
:108A20000BE0204600F078FA07E02046F8F716FD44
:108A300002E02046FBF7E6F9009001208AF80000EA
:108A400042E02046FEF7D6FB6CE72046FCF786FEA8
:108A5000039039E02046FCF7D1FC02E02046FDF708
:108A60000DF8019030E02046FDF7CCF9F9E7000061
:108A7000EC010020A4370020002400200C0300207B
:108A80000010014002000020AA555AA5140300203E
:108A90006C2B0020002900202046FDF7F5FAE0E7C6
:108AA0002046FDF733FCDCE72046FDF771FDD8E7F3
:108AB0002046FDF7AFFED4E72046FDF7EDFFD0E7F7
:108AC0002046FEF7B3FB02907889132806D0019860
:108AD00038B10020A2469425019013E0DFF89CA055
:108AE00038E0029820B10020A2466025029009E0FB
:108AF000039810B30020039084F8E86084F8E960DC
:108B0000A246EA250020009029465046FBF758F976
:108B1000020A0AF805200AEB05010022487010211C
:108B20001748FAF70EF8502001F00EF8AA1C51462B
:108B30001448FAF7FAFF134D11E0009820B184F8B9
:108B40003C6084F83D6004E0FF2084F83C0084F839
:108B50003D00A2463E25D5E7012001F0F9FA95F83F
:108B600039002128F8D0502000F0EEFF012210211A
:108B70000348F9F7E6FFC8F8006096E500290020F1
:108B8000000801406C2A0020DFF874801D4F1E4E43
:108B90001E4DDFF87CB04FF4806A51465846F9F715
:108BA000C8FFF7F7F5FD002425E0052C0FD2DFE81C
:108BB00004F00E0306090C00134E144D07E0154E89
:108BC000154D04E0154E164D01E0164E164D04EB02
:108BD0008409234658F839002A463146F7F7B6FF8C
:108BE00008EBC90188612046F8F746FA642001F0D5
:108BF000AFFA641CE4B23888A042CED9D5E70000B1
:108C0000A03E0020A83600208403002070C4000885
:108C1000001001401405002000C60008A406002032
:108C200090C700083408002020C90008012001F086
:108C30008FFAFBE7012001F08BFAFBE7012001F03E
:108C400087FAFBE7012001F083FAFBE7012001F03E
:108C50007FFAFBE7012001F07BFAFBE70B4E0A4CA1
:108C6000DFF82C804FF4FA753715284601F070FABA
:108C7000A0690121401CA0613046F9F75AFF39462E
:108C80004046F9F756FFF0E70800002000080140D1
:108C9000001001402DE9F843304F4FF480644FF04D
:108CA000AA3821463846F9F744FF02222C49684683
:108CB000F8F784FBBDF80000294D0104BDF802005F
:108CC0007A3D0843274E404506D0B0F1BB3F43D024
:108CD0002549C84240D127E0A14621463846F9F748
:108CE00028FF002004464219210292F8BE40401C91
:108CF0000C430428F7D3DFF8748021464046F7F789
:108D000039FE78B122464146304600F03BFF4946E5
:108D10003846F9F70EFF12491148022284314430D7
:108D2000F8F75AFBFEF766FC002001460A024119DB
:108D3000401C91F8FE1011430428F7D3B1F5003F11
:108D40000AD23046F7F716FE002805D0002080F33F
:108D50001388304600F000FFBDE8F88300100140A2
:108D60007AF00708000002084544AAAA0000040897
:108D700010B5502080F31188BFF34F8FBFF36F8F72
:108D800002F032FE18B104494FF080500860002014
:108D900080F3118810BD000004ED00E030B58FB005
:108DA00028216846F7F761FA14210AA8F7F75DFA57
:108DB00001210804CDE90010002402940225049149
:108DC000CDE907504FF4E01009906846FAF788F8AB
:108DD00008B172B6FEE70F20CDE90A054FF48060B6
:108DE000CDE90C4002210AA80E94F9F76DFF002886
:108DF00001D072B6FEE70FB030BD70470148FAF7F8
:108E00002FBB00005C2900200148FAF729BB0000B5
:108E1000A42900200148FAF723BB0000402D0020C0
:108E2000F0B502681C4B1D4D1D4E1E4F1E4C4FF0E1
:108E3000804C984209D0A04207D0604505D0A84296
:108E400003D0B04201D0B84204D122F0700E4A687B
:108E500042EA0E02984209D0A04207D0604505D0F0
:108E6000A84203D0B04201D0B84203D122F44075E9
:108E7000CA682A434D6922F080022A4302608A6848
:108E8000C2620A688262984201D0A04201D1096997
:108E9000016301214161F0BD002C0140000400404C
:108EA00000080040000C00400034014010B5846808
:108EB00042EA032224F47F440A432243826010BD25
:108EC000826822F070020A4342F007018160704715
:108ED00010B5036A046A24F001040462846924F072
:108EE000F00444EA021423F00A020A438461026295
:108EF00010BD10B5036A23F0100303628369046A8E
:108F000023F4704343EA023224F0A00343EA011140
:108F10008261016210BD00002DE9F05F04463F4808
:108F20003D4E4FF6FF77817CC27C07EA0121334634
:108F30000A430025DFF8E8801B7DDFF8E8A04FF04A
:108F4000010C00F1160104F1160B4FF49679012A79
:108F50002FD0002A2BD13288002A28D1062B26D1E7
:108F6000A6F800C0027D07EA0223427D2E481A437C
:108F7000A8F80020F7F760F90027D046D8F80000DD
:108F800008B1308840B1012001F0E2F87F1C4F4564
:108F9000F4DBD8F80000D8B3244825490268100A49
:108FA000207562755846F7F747F9C8F80050BDE8D4
:108FB000F09F7288002AFAD1062BF8D1A6F802C0D9
:108FC000027D07EA0223427D1A481A43A8F80020CE
:108FD000F7F732F9DFF86080002700BFD8F800000B
:108FE00008B1708840B1012001F0B2F87F1C4F45F4
:108FF000F4DBD8F8000058B1104811490268100A93
:10900000207562755846F7F717F9CAF80050CEE791
:10901000FFE725756575CAE7A43700200024002006
:10902000C409002008030020183700201C0300207A
:10903000FC0E00205E3700201003002018030020E3
:1090400000280020F0B58BB005461B4E1B4C282194
:109050006846F7F70AF9B4F81D00ADF80000207D66
:10906000174F062804D1012239466846F8F7B4F9AB
:10907000012239466846F8F7A1F9BDF80000000A58
:109080006874BDF800002874BDF80000A0F57F41A9
:10909000FF3901D0A6F86600287C617F884206D19E
:1090A000687CA17F884202D1207D062802D0002062
:1090B0000BB0F0BD0120FBE7A8360020A43700204C
:1090C00048F0070810B501F065FE002805D0D0E98A
:1090D0000021BDE810400846104710BD10B5406A99
:1090E0000021C185C184FAF7A8FA10BD70B5446AA1
:1090F0002068406994F83910C0F3C0100025212978
:1091000004D118B1E584204600F046F82068406993
:1091100094F83A10C0F38010222904D118B1E585E3
:10912000204600F02BF8E06B40F01000E063204692
:10913000FAF783FA70BD10B50146406A09680968FC
:10914000890613D40021C1850168CA6822F480729F
:10915000CA6001684A6922F001024A6101684A69ED
:1091600022F040024A61202180F83A10FAF782FC8E
:1091700010BD10B5406AFAF77EFC10BD0168CA68E0
:1091800022F49072CA6001684A6922F001024A61C1
:10919000202180F83A1070470168CA6822F0C002A6
:1091A000CA60202180F83910704710B590F83A1045
:1091B000222901D0022010BD82684FF480539A42C8
:1091C00001D1016921B1816A9A421BD04AB10AE0FA
:1091D0000268816A5268C2F308020A80816A891CA7
:1091E00008E0026972B10268526802F07F020A70F8
:1091F000816A491C8162C18D491E0904090CC1851F
:1092000003D016E002685268F1E70168CA6822F0EC
:109210002002CA600168CA6822F48072CA600168CC
:109220004A6922F001024A61202180F83A10FAF7D7
:1092300021FC002010BD000070B5044600680169E3
:10924000E26821F44051114301612169A06808439B
:10925000616908432168CA6841F20C639A4302437A
:10926000CA6020684169A26921F4407111434161DB
:109270001E492068884202D1F9F7ECFD01E0F9F7B8
:10928000D9FD00EBC00101EB001260686421800091
:10929000B2FBF0F3B3FBF1F36FF018067343B2FBCC
:1092A000F0F5B2FBF0F605EB8305322303EB051571
:1092B000B5FBF1F5B6FBF1F605F0F00505EB06158B
:1092C000B2FBF0F6B2FBF0F0B0FBF1F06FF0180279
:1092D000504306EB800003EB0010B0FBF1F0216877
:1092E00000F00F002844886070BD00000038014085
:1092F00090F83910212901D0022070478168B1F51A
:10930000805F01D10169E1B1016A4A1C0262026811
:1093100009785160C18C491E0904090CC18404D02C
:10932000C18C4FF6FA72914209D90168CA6822F0DD
:109330008002CA600068C16841F04001C16000203D
:109340007047016A02680988C1F308015160016A27
:10935000891C0162DEE72DE9F041984617460E466A
:109360000446069D1DE0681C1BD02DB1F9F7EEFBED
:10937000A0EB0800A84214D92068C16821F4D0717C
:10938000C1602068416921F001014161202084F819
:10939000390084F83A00002084F838000320BDE842
:1093A000F0812068006836EA000004D00020B8424E
:1093B000D9D00020F3E70120F9E7000038B51248C2
:1093C00000680168C943C90618D401684068009064
:1093D0000D48FAF706F90D48006840680C4CC0F5D6
:1093E00080720C490C486261F6F726FF4FF48072D8
:1093F00008490548FAF7F2FA01202060BDE8384034
:109400000148FAF71BB900002C2A0020302C00205C
:1094100008030020BC0C0020FC0E002038B51248C8
:1094200000680168C943C90618D401684068009003
:109430000D48FAF7D6F80D48006840680C4CC0F5A6
:1094400080620C490C48E260F6F7F6FE4FF4806249
:1094500008490548FAF7C2FA01206060BDE83840C3
:109460000148FAF7EBB800006C2A0020B82C002065
:1094700008030020002000200024002038B51148F7
:10948000FAF7DCF80F4800680168C943C90618D428
:109490000168406800900B48FAF7A3F80A48006892
:1094A00040680A4CC0F5807209490A482261F6F703
:1094B000C3FE4FF4807206490248FAF78FFA012082
:1094C000A06038BDAC2A0020FC2C0020080300203E
:1094D000BC0D002000280020FEE7000070B58AB017
:1094E0001B4D28216846F6F7C0FE002401221949C9
:1094F0006846F7F763FFBDF800004FF6FF76B0420D
:1095000000D0A880082214496846F7F757FF68463C
:1095100009E000BF30F81410B14202D005EB44025C
:109520009182641CE4B22988A142F3D800200B493F
:1095300008E000BF05EB40020B88928A401C1A44E9
:109540000A80C0B22A888242F4D80AB070BD0000F6
:10955000A836002028F0070800E007084C03002088
:10956000114810B5418811B9017D062901D00020AC
:1095700010BD0D4C01214180463C807F20700620AB
:10958000607000200222A070E2702071617120469C
:109590000621FAF715FC010AA1710449E0710820BF
:1095A0000880012010BD0000A4370020C40900205D
:1095B000124810B5418811B9017D062901D000205B
:1095C00010BD0E4C01214180463C817F2170062157
:1095D00061700021A1701021E170C17F217190F8AC
:1095E0002000607120460621FAF7EAFB010AA1710A
:1095F0000349E07108200880012010BDA437002035
:10960000C40900202DE9F0418AB007462B4E2C4CAE
:1096100028216846F6F729FE00206D4605E021184E
:10962000497F25F81010401CC0B2217E8142F6D837
:10963000207DDFF89080062804D10122414628468B
:10964000F7F7CAFE012241466846F7F7B7FEBDF8B4
:1096500000003874BDF80000052800D2B080207DDD
:10966000DFF86480062804D108224146A81CF7F7D9
:10967000B3FE08224146A81CF7F7A0FE002013E025
:1096800005EB4002231851889B7F994202D0237D2D
:10969000062B10D0082905D206EB40039982917859
:1096A0003A185174401CC0B2217E8142E8D8012092
:1096B0000AB0BDE8F0810020FAE70000A8360020DB
:1096C000A437002028F0070800E00708C0B210B552
:1096D000264900EB001000EB4000244C31F810301C
:1096E0000122002104EB4000012B01D07BB11CE0E2
:1096F000A0F85210B0F850305B1C9BB2A0F850306C
:10970000022B12D3A0F85010A0F858200DE0A0F8BA
:109710005010B0F852305B1C9BB2A0F85230022BB4
:1097200003D3A0F85210A0F85810038D012B0FD0CE
:10973000002B0CD1A0F85410B0F85620521C92B255
:10974000A0F85620022A02D320F8561F818010BDAF
:10975000A0F85610B0F854305B1C9BB2A0F85430FF
:10976000022BF4D320F8541FC28010BD3E380020D5
:109770000FB4084B10B504A902AA039800F03EF8F4
:10978000044602A9002000F0DAF9204610BC5DF87A
:1097900014FB00003F9B00080907090E002804DBAA
:1097A00000F1E02080F80014704700F00F0000F195
:1097B000E02080F8141D7047BFF34F8F0548016803
:1097C000054A01F4E06111430160BFF34F8F00BF10
:1097D000FDE700000CED00E00400FA0502E008C817
:1097E000121F08C1002AFAD170477047002001E01B
:1097F00001C1121F002AFBD1704700002DE9FF4F65
:109800008BB088460546002606E025280BD0DDE90A
:109810000D1290476D1C761C28780028F5D10FB0EA
:109820003046BDE8F08F0024A146A2460122AE4991
:1098300000E0044315F8013F203B02FA03F0084220
:10984000F7D128782A2810D06FF02F022878A0F1BD
:109850003001092915D809EB890102EB410144F0D7
:10986000020400EB01096D1CF0E758F8041B5FEAE5
:10987000010903D544F40054C9F1000944F002047D
:109880006D1C28782E2817D115F8010F44F0040418
:109890002A280ED06FF02F022878A0F13001092974
:1098A0000AD80AEB8A0102EB410100EB010A6D1CA8
:1098B000F2E758F804AB6D1C28786C280FD006DC52
:1098C0004C2817D068280DD06A2814D104E07428D9
:1098D00010D07A280FD10DE044F400140AE044F4CB
:1098E000801401E044F440146978814202D104F507
:1098F00080146D1C6D1C2878692865D006DC002852
:109900008DD0632827D0642806D15DE06E2808D06A
:1099100073282AD0752877D0DDE90D129047761C80
:10992000E0E0C4F30250022809D003280DD0D8F893
:10993000001004280DD00E6008F10408D2E0D8F819
:109940000010F217C1E90062F6E7D8F800100E80A7
:10995000F2E70E70F0E718F8041B8DF800100020F5
:109960008DF80100EB46012003E058F804BB4FF0EE
:10997000FF3061074FF0000701D40AE07F1C574514
:109980000DDA8742FADB1BF807100029F6D106E052
:109990007F1C8742FCDB1BF807100029F8D1DDE9AA
:1099A0000D23A9EB07008146214600F0B1F83044B1
:1099B000C61904E0DDE90D121BF8010B90477F1E6C
:1099C000F8D22146484688E058F8040BC4F3025107
:1099D0004FF00A0B032900D100B2042900D140B294
:1099E000002802DA40422D2102E0210505D52B2175
:1099F0008DF82410012104E006E0E10710D02021B9
:109A0000F6E708AF089113E058F8040BC4F30251CD
:109A10004FF00A0B032900D180B2042900D1C0B253
:109A20000021EEE75946F6F735FD303107F8011D04
:109A30000028F7D1ADEB070000F1200B600702D53D
:109A400024F4803401E04FF0010ADA4502DDAAEB8C
:109A50000B0000E00020824600EB0B010898014457
:109A6000A9EB01000A90E00306D4DDE90D232146AD
:109A70000A9800F04DF806444FF0000908E009A9E3
:109A800011F80900DDE90D12904709F10109761C72
:109A900008998945F3DBE0030CD5DDE90D23214668
:109AA0000A9800F035F8064404E0DDE90D12302094
:109AB0009047761CBAF10001AAF1010AF5DC05E035
:109AC000DDE90D1217F8010B9047761CBBF1000180
:109AD000ABF1010BF4DC0A982146DDE90D2300F01F
:109AE00005F806446D1C97E6092801002DE9F041B0
:109AF000044600251E461746880404D405E039466E
:109B00002020B0476D1C641EF9D52846BDE8F081C1
:109B10002DE9F041044600251E469046C80301D5B4
:109B2000302700E02027880404D505E04146384668
:109B3000B0476D1C641EF9D52846BDE8F0810A685F
:109B4000531C0B6010707047C100002001E000BF83
:109B5000401C8842FBD3704710B5084A0168114089
:109B6000B1F1005F09D1064C4168A1610068F6F7C8
:109B7000EBFAA069BDE81040004710BD0000FE2FC1
:109B8000CC0900202DE9F05F0024904606460D46E2
:109B900027464FF48069DFF854A0DFF854B018E08E
:109BA000687815F8021B01EB00202AF81400641CE9
:109BB000A4B2484684420BD1014600245846F8F727
:109BC000B8FF4A4609493046FDF792FB06F50066A4
:109BD000BF1C4745E4D3002C06D022463046BDE8E2
:109BE000F05F0249FDF784BBBDE8F09F42580020BA
:109BF0000010014086B00024009401940294039464
:109C0000FFF748F8F8F7B0FFF7F744F8FBF79AF9D1
:109C1000FFF764FCF6F7F4FEFFF7C0F8FAF7B4FDBF
:109C2000FE48416941F001014161416901F00101D2
:109C30000491416941F0020141614069002200F054
:109C40000200049005210E20F9F70CF80E20F8F719
:109C5000FBFF002205213B20F9F704F83B20F8F731
:109C6000F3FFFAF7C1FEEF48ED4901604FF4E1312F
:109C7000C0E901140C21C460C0E904418461C461DD
:109C8000F9F766FD08B172B6FEE7FAF7D5FEFAF706
:109C9000FBFEE649E44808600846F8F785FA08B193
:109CA00072B6FEE7DF490494A439E14805940860E0
:109CB0000846F8F7C6FA08B172B6FEE73C20CDE9CF
:109CC0000404D848102204A9A438F8F793FA08B17C
:109CD00072B6FEE7FAF720FEFAF754FEFAF7D8FD5F
:109CE0000122D44E550329463046F8F72AFF0122B7
:109CF000170339463046F8F724FFDFF83C8301228A
:109D000010214046F8F71DFFE81000900120CDE932
:109D10000104022003906946C848F8F709FE0022B2
:109D200029463046F8F70DFF002229463046F8F75D
:109D300008FF002239463046F8F703FF00221021C1
:109D40004046F8F7FEFE0220F8F72EFD2021BC4821
:109D5000F6F78BFA0522BBA1B948FFF709FDB84910
:109D600082B24FF49673A1F18000F9F785FE0122CB
:109D700029463046F8F7E5FE012239463046F8F725
:109D8000E0FE012210214046F8F7DBFE00F01CFA4D
:109D9000B14800F08FFAA54CD83C6061AE48103055
:109DA00000F088FAA061AC48203000F083FAE0614E
:109DB000A948303000F07EFA2062A748403000F019
:109DC00079FA6062A448503000F074FAA062A248A8
:109DD000603000F06FFAE0629F48703000F06AFA7D
:109DE00020639D48803000F065FA60639A489030A7
:109DF00000F060FAA0639848A03000F05BFAE063DE
:109E00009548B03000F056FA934A01212064C032E0
:109E1000084600F08FFA904A01216064D03208466B
:109E200000F088FA8C4A0121A064E032084600F074
:109E300081FA894A0121E064F032084600F07AFA9A
:109E400001212065854A084600F074FA834A012101
:109E500060651032084600F06DFA804A0121A06565
:109E60002032084600F066FA7C4A0121E065303273
:109E7000084600F05FFA794A02212066403208461F
:109E800000F058FA754A022160665032084600F028
:109E900051FA724A0221A0666032084600F04AFA7E
:109EA0006E4A0221E0667032084600F043FA6A4BBF
:109EB0002067A03B00220121694800F0E5FAA4F1E7
:109EC0008005654BE866903B00220121654800F063
:109ED000DBFA614B2867803B00220121624800F0D9
:109EE000D3FA5D4B6867703B002201215F4800F0A8
:109EF000CBFA594BA867603B002201215C4800F077
:109F0000C3FA554BE867503B00220121594800F045
:109F1000BBFA514B2060403B00220121564800F023
:109F2000B3FA4D4B6060303B00220121534800F0F2
:109F3000ABFA494BA060203B00220121504800F0C1
:109F4000A3FA454BE060103B002201214D4800F090
:109F50009BFA20614C4A0221102000F071F94A4A14
:109F6000686518320221102000F06AF9464AA86597
:109F700030320221102000F063F9434AE86548328C
:109F80000221102000F05CF93F4A2866603202216D
:109F9000102000F055F93C4A686678320221102002
:109FA00000F04EF9A866394A0021394800F01AFA43
:109FB000364A686224320021364800F013FA334AE8
:109FC000A86248320021344800F00CFA2F4AE862B7
:109FD0006C320021314800F005FA2C4A2863903297
:109FE00000212F4800F0FEF9284A6863B4320021AE
:109FF0002C4800F0F7F9244AA863D83A00212A48EF
:10A0000000F0F0F9204AE863B43A0021274800F054
:10A01000E9F91D4A2864903A002149E00010024005
:10A0200000500040EC290020003002406001002078
:10A0300000740040000C0140000801400010014085
:10A04000EC2A00207379737974656D2072657365ED
:10A05000742E2E2E2535640070C2000870C30008CF
:10A06000810C0008850C0008870C0008890C00088A
:10A070008B0C00088D0C00088F0C0008910C000858
:10A08000930C0008830C000840C1000890BF000832
:10A09000557600085D760008B57B00088D860008BF
:10A0A000898B00082D8C0008358C00083D8C000839
:10A0B000214800F097F96864204A0021204800F008
:10A0C00091F91E4AA864243200211E4800F08AF942
:10A0D0001A4AE864483200211B4800F083F92865D9
:10A0E0001A4800F04FF860671848103000F04AF83E
:10A0F000A0671648203000F045F8E067134830307C
:10A1000000F040F8803420601048403000F03AF809
:10A1100060600E48503000F035F8A0600B486030A9
:10A1200000F030F8E0600948703000F02BF8206152
:10A1300000F066F8FEE70000458C0008D4C0000877
:10A140004D8C0008558C00085D8C0008F0C3000899
:10A1500010B5EFF3058149B9EFF3108131B9084922
:10A160000968022905D1EFF3118111B16FF00504DF
:10A1700003E0002408B100F08FFF204610BD00006E
:10A18000940A002010B54FF00001EFF30582BAB930
:10A19000EFF31082A2B90B4A1268022A02D1EFF340
:10A1A00011826AB948B1D0E902202AB1202807D328
:10A1B000104601F065F802E010B901F053F80146CD
:10A1C000084610BD940A0020EFF3058058B9EFF35C
:10A1D000108040B909490868022801D030B109E06F
:10A1E000EFF3118030B16FF0050070470120086077
:10A1F000002070474FF0FF3070470000940A0020A5
:10A2000010B5EFF3058060B9EFF3108048B90B4942
:10A210000868022802D0012806D00BE0EFF3118075
:10A2200040B16FF0050010BD0220086000F09CFFF7
:10A23000002010BD4FF0FF3010BD0000940A002038
:10A24000F8B514464FF00005EFF305826ABBEFF353
:10A25000108252BB164A1268022A02D1EFF3118211
:10A260001ABB10B309B3ACB1D4E902326BB1502AB6
:10A270001BD32269CAB1676900FB01F6B74214D348
:10A280000025009501F0DFF807E072B9226962B994
:10A29000626952B9002201F0B2F8050005D00CB194
:10A2A000216800E0002100F095FE2846F8BD00007E
:10A2B000940A002070B505464FF00004EFF30580C6
:10A2C000A0BBEFF3108088BB19480068022802D1B8
:10A2D000EFF3118050BB0DB1686800E00020C107AA
:10A2E00001D0012600E0002600071FD46DB1D5E99A
:10A2F000021021B1502819D31EB1042002E020B170
:10A3000014E0012001F06EF805E00EB1042000E039
:10A31000012001F05CF8040008D00DB1296800E0CC
:10A32000002100F057FE0EB144F00104204670BD3C
:10A33000940A0020F8B5144603460E464FF0000577
:10A34000EFF30580E8BBEFF31080D0BB2448006832
:10A35000022802D1EFF3118098BB93B39E423DD8FF
:10A360004CB1A0680028E06803D0502836D3012003
:10A3700002E008B132E00020012B05D010B31846EE
:10A38000A26801F004F820E040B103200090002210
:10A3900011460120A36801F056F804E003220021D1
:10A3A000012001F02CF8050018D086B100231A46D0
:10A3B000194601F0BFF8012809D0284600F01EFE1A
:10A3C00000250BE0184600F0C5FF050006D00CB1D3
:10A3D000216800E00021284600F0FCFD2846F8BD79
:10A3E000940A0020F0B585B04FEA01034FF0000455
:10A3F000EFF305810394A1BBEFF3108189BB2149E1
:10A400000968022902D1EFF3118151BB48B38026BC
:10A4100018218DF8104004AD42B3176807B13D46CE
:10A4200097691FB139467F1E382F02D21779FF076F
:10A4300002D0002005B0F0BD576907B1BE08D2F8C0
:10A4400008C0BCF1000F0DD0D4685C2C18D3126981
:10A450003AB137B18DE806103246294601F085FA47
:10A4600003900DE0D7685FB912694AB903AACDE934
:10A470000012B2B2294601F04BFA012800D0039431
:10A480000398D7E7940A00202DE9FC411C461746A3
:10A49000884606464FF00005EFF3058078BBEFF3E2
:10A4A000108060BB17480068022802D1EFF31180CA
:10A4B00028BB26B3082000F001FC03001FD0B8F130
:10A4C000000FC3E9006711D001220F4E00208CB1AC
:10A4D000216801B10846A16851B1E468302C0ED35F
:10A4E000CDE90061012101F0D7FB07E00022ECE794
:10A4F000E16821B90121009601F0B4FB0546284628
:10A50000BDE8FC81940A0020C59000082DE9F041C7
:10A51000154C0F46054666692168002081F85A00EF
:10A520002068001D00F05AFC681C07D137B1216873
:10A53000BDE8F0410D48091D00F0A1BC206835447C
:10A54000B5424560216805D2A068BDE8F041091D0B
:10A5500000F07DBC6068091D00F079FC206B85422D
:10A5600000D22563BDE8F081440A00205875002020
:10A570002DE9F041054600F08FFC2D4C2069401C70
:10A58000206120682B4F10B1E06930B32BE02560CB
:10A590002069012827D1002606EB860007EB800002
:10A5A00000F047FC761C382EF6D3234800F041FC1F
:10A5B0002148143000F03DFC1F48283000F039FCE1
:10A5C0001D483C3000F035FC1B48503000F031FC99
:10A5D000194860601430A06005E02068E96AC06A2C
:10A5E000884200D82560E06A401CE0626864E86A3E
:10A5F000A169884200D9A06100EB800007EB8000D0
:10A60000291D00F03CFC00F067FCE06900280CD03C
:10A610002068E96AC06A884207D208494FF0805032
:10A620000860BFF34F8FBFF36F8FBDE8F08100006C
:10A63000440A0020A87000200875002004ED00E006
:10A6400038B500F029FC104CA068C8B90F4800F0DC
:10A65000F0FB0E48143000F0ECFB0C482060143086
:10A6600060600A4B00202833009003F15002102153
:10A670000A2000F0E8FEA06010B105A100F0AAFCDD
:10A68000BDE8384000F028BC800A00206C7500202E
:10A69000546D72510000000030B4026C0B46002A69
:10A6A0000BD0C1681144C1604468A14201D3016864
:10A6B000C16030BC1846F5F7BFBD30BC70472DE90E
:10A6C000F041856B174604460026026C82B1C7B183
:10A6D000E068F5F7B1FDE168206C091AE1602268D5
:10A6E000914202D26168081AE060022F16D017E08A
:10A6F0002068A8B9606801F0DBF9064600206060B8
:10A700000EE0A068F5F798FD216CA0680844A060F1
:10A710006168884204D32068A06001E005B16D1E25
:10A720006D1CA5633046BDE8F08110B5044690F875
:10A73000590058B101280CD002280FD0502080F3C6
:10A740001188BFF34F8FBFF36F8FFEE7206B00F0D0
:10A75000D7FB2046BDE8104000F0D2BB10BD000082
:10A7600010484FF48041420706D0C01D0D4920F02B
:10A770000700411AC1F580410B4A00230144C2E998
:10A7800000030839103A21F0070111604B600B609B
:10A790000B1AC0E9001393604FF000405360D06083
:10A7A000704700003C7D0020A80A0020154E164C82
:10A7B000A6F29C474FF08058DFF8509012E000BF9F
:10A7C00000F06AFBF068C568281D00F007FB2069EF
:10A7D000401E2061E068401EE06000F07DFB2846DE
:10A7E000FFF7A3FFE0680028EAD13868012805D9FF
:10A7F000C9F80080BFF34F8FBFF36F8F00F018FBD5
:10A80000F0E7000044750020440A002004ED00E059
:10A81000002807D00021416001600B460A46C16054
:10A8200000F088BE7047000070B51D46049C51B111
:10A83000C4F80020C4E90F010121204600F036FED3
:10A8400084F84C5070BD2460F4E72DE9F0470E46C3
:10A85000DDE909841746824691009946089DA522A4
:10A86000206BF5F7FBFC6FF00301206B01EB870118
:10A87000084420F00707780707D0502080F311889C
:10A88000BFF34F8FBFF36F8FFEE72218315C82F862
:10A890003410315C11B1401C1028F6D3002684F826
:10A8A0004360382D00D33725E562C4E91356201DD7
:10A8B00000F0CAFA04F1180000F0C6FA2461C5F1EC
:10A8C00038006462A061666584F8586084F85A6054
:10A8D0004A465146384600F06FFA2060B8F1000F42
:10A8E00001D0C8F80040BDE8F0872DE9F0471E46CA
:10A8F000DDE9089417460D0080460ED0002C14D0D8
:10A90000FFF79EFEC4F80080C4E90657C4E9086951
:10A91000201DBDE8F04700F097BA502080F3118861
:10A92000BFF34F8FBFF36F8FFEE7BDE8F0870000E6
:10A9300030B5114900E011460A688242FBD34B68EA
:10A940005C18844203D14068184448600846436854
:10A950001C18944209D1084C103C2468A24209D02A
:10A9600052681A4442600A6812680260814200D04C
:10A97000086030BD0460F9E7A80A002070B5002423
:10A9800041600B4D0061914206D8D11A8269914213
:10A9900006D2011D686807E09A4203D2994201D3AA
:10A9A000012403E0011D286800F051FA204670BD23
:10A9B000800A002010B5044600F06EFAA06B28B1A2
:10A9C0005FF0000400F088FA204610BD0124F9E78A
:10A9D00030B589B0304D55E00498002806DADDE93D
:10A9E0000601059A9047049800284BDB069C606995
:10A9F00010B1201D00F0F2F902A800F0B9F80246EB
:10AA000004980A283ED2DFE800F00505053D263708
:10AA100005053D260598A169034601442046FFF738
:10AA2000ADFF00B3616A20468847E069012829D15B
:10AA3000002000900598A16900234218194620467D
:10AA400001F072F978B9502080F31188BFF34F8F6D
:10AA5000BFF36F8FFEE70598A06128B181181346F8
:10AA60002046FFF78BFF0DE0502080F31188BFF3E5
:10AA70004F8FBFF36F8FFEE794F82C0010B920467C
:10AA800000F03EFA002204A9A86800F061FE002848
:10AA9000A2D109B030BD0000800A00202DE9FC41A0
:10AAA0000F46054600F0A4FB01A800F061F804463B
:10AAB000019818B101F074F8BDE8FC81224EAFB1E5
:10AAC00070680068A8B30027291B3A46B06800F0F8
:10AAD000C1FA01F065F80028EED11C494FF0805012
:10AAE0000860BFF34F8FBFF36F8FE5E7A542EBD848
:10AAF00001F056F830682746C068C468201D00F091
:10AB00006DF9E069012810D1A0692B4641193A4638
:10AB10002046FFF733FF40B1002003460146009076
:10AB20002A46204601F000F920B1616A2046884794
:10AB3000C2E707E0502080F31188BFF34F8FBFF3C7
:10AB40006F8FFEE70127BFE7800A002004ED00E0D9
:10AB500006484168096829B14168C968C9684968F7
:10AB6000016370474FF0FF31FAE70000440A00200C
:10AB700070B5054600F032FF064E04463069844247
:10AB800003D200F009F8012000E0002028602046F0
:10AB9000346170BD800A0020F8B5194D1FE0C0680F
:10ABA000C4680668201D00F019F9616A20468847CC
:10ABB000E069012813D1A0693044B04206D924616C
:10ABC0006060211D286800F042F908E0002003467B
:10ABD000014600903246204601F0A6F838B12868B8
:10ABE00001680029DBD16968C5E90010F8BD502073
:10ABF00080F31188BFF34F8FBFF36F8FFEE7000024
:10AC0000800A002008484068401C4FF0500080F344
:10AC1000118804D0BFF34F8FBFF36F8FFEE7BFF3F0
:10AC20004F8FBFF36F8FFEE7B00A0020074C2068FC
:10AC3000016841B1C0680021D0F80000FFF72EFF85
:10AC4000FFF7C6FEF3E701210020F7E7800A0020A6
:10AC50002DE9F041044600F01FF994F9455004F144
:10AC6000240609E0606A48B1304600F061FF08B18F
:10AC700000F040FA6D1E6DB2002DF3DC4FF0FF3690
:10AC800084F8456000F028F900F006F994F9445082
:10AC900004F1100709E0206948B1384600F048FF88
:10ACA00008B100F027FA6D1E6DB2002DF3DC84F8B8
:10ACB0004460BDE8F04100F00FB900002DE9F0411B
:10ACC0000546002700F094FA314E306808B9FFF7C6
:10ACD00047FDF06805424BD1C5B3083568070ED073
:10ACE00005F00700C0F108000544680707D05020B0
:10ACF00080F31188BFF34F8FBFF36F8FFEE72DB343
:10AD00007068854234D82248103001460C6801E052
:10AD100020460C466168A94202D221680029F7D179
:10AD200031688C4224D00768216801606068083768
:10AD3000411B10290FD96019420708D0502080F319
:10AD40001188BFF34F8FBFF36F8FFEE710E04160B4
:10AD50006560FFF7EDFD61687068401A7060B26869
:10AD6000904200D2B060F06801430020C4E90001C5
:10AD700000F016FF780707D0502080F31188BFF34A
:10AD80004F8FBFF36F8FFEE73846BDE8F0810000BC
:10AD9000980A002010B5040006D000F07DF8246A5F
:10ADA00000F09AF8204610BD502080F31188BFF3C0
:10ADB0004F8FBFF36F8FFEE710B5031F4FF0807406
:10ADC0001C601B1F21F001011960191F024B0B6051
:10ADD000143940380A6010BD05AC0008D0E90132D2
:10ADE00001699A60D0E901235A604A68824201D120
:10ADF00082684A60002202610868401E0860086894
:10AE000070470000034B036003F15C000860802082
:10AE10001060704784760020044B036003F15C00EF
:10AE200008604FF48070106070470000E0780020E8
:10AE3000704700F108014FF0FF32C0E90112C16014
:10AE4000016100210160704700210161704730B548
:10AE50000B685A1C02D000F1080202E0026904E00B
:10AE60002246546825689D42FAD953684B60996020
:10AE70008A60516008610168491C016030BD426808
:10AE80004A6093688B6093685960916008610168BB
:10AE9000491C016070470000502080F31188BFF307
:10AEA0004F8FBFF36F8F0A494868401C48600128E4
:10AEB0000CD10848006810F0FF0F07D0502080F335
:10AEC0001188BFF34F8FBFF36F8FFEE7704700000D
:10AED000B00A002004ED00E00849486828B1401E8F
:10AEE000486001D180F311887047502080F31188A9
:10AEF000BFF34F8FBFF36F8FFEE70000B00A002053
:10AF000070B5002827D0144DA0F108046168E868E6
:10AF1000014207D1502080F31188BFF34F8FBFF358
:10AF20006F8FFEE722683AB1502080F31188BFF39B
:10AF30004F8FBFF36F8FFEE78143616000F058F9D8
:10AF400060686968084468602046FFF7F1FCBDE866
:10AF5000704000F025BE70BD980A00204FF0E02040
:10AF600000210161816105494FF47A720968B1FBE2
:10AF7000F2F1491E4161072101617047340A002046
:10AF800010B5F5F72DF9114910280ED300F1E02086
:10AF900090F8F0030A78904207D2502080F311888D
:10AFA000BFF34F8FBFF36F8FFEE7094800688968D2
:10AFB00000F4E060884207D9502080F31188BFF385
:10AFC0004F8FBFF36F8FFEE710BD0000B00A002067
:10AFD0000CED00E010B5084B002200BF53F83240E2
:10AFE0001CB1521C082AF9D310BD43F8321003EBF0
:10AFF000C201486010BD00006870002010B5040058
:10B000000AD000F013F894F8460000280CD120462E
:10B01000BDE81040FFF774BF502080F31188BFF3E4
:10B020004F8FBFF36F8FFEE710BD0000084A00216D
:10B0300002EBC1035B68834206D1002042F8310075
:10B0400002EBC10148607047491C0829F0D37047E2
:10B050006870002070B515460E460446FFF71CFFC9
:10B0600094F944100020491C01D184F8440094F95B
:10B070004510491C01D184F84500FFF72DFFA06B56
:10B0800028B92A46314604F1240000F051F8204640
:10B09000BDE87040FFF7DCBD10B5020014D00F48CA
:10B0A000806B38B1502080F31188BFF34F8FBFF30E
:10B0B0006F8FFEE700F09CF800211046FFF726FA9C
:10B0C00000F06EFD002807D105494FF08050086060
:10B0D000BFF34F8FBFF36F8F10BD0000440A0020F5
:10B0E00004ED00E002498A6A0260496941607047E4
:10B0F000440A00200149012048627047440A0020A8
:10B1000010B50C4650B1094909681831FFF79FFE88
:10B110002046BDE810400121FFF7F8B9502080F328
:10B120001188BFF34F8FBFF36F8FFEE7440A0020F3
:10B1300070B514460D4668B10A4909681831FFF721
:10B140009EFE0CB14FF0FF3521462846BDE8704009
:10B15000FFF7DCB9502080F31188BFF34F8FBFF3A6
:10B160006F8FFEE7440A002030B587B000240394B7
:10B1700005AA04A903A80494FFF744FEDDE903012E
:10B180000094CDE90110002315A11748059A00F09D
:10B19000ECFB164D002868631FD000F095FD0128D8
:10B1A00009D0401C19D1502080F31188BFF34F8F74
:10B1B000BFF36F8FFEE7502080F31188BFF34F8FEE
:10B1C000BFF36F8F4FF0FF3028630120E8616C619F
:10B1D00007B0BDE8304000F069B807B030BD0000EE
:10B1E00049444C4500000000ADA70008440A002077
:10B1F0000248816B491C816370470000440A0020AB
:10B20000164810B5816B11B10121416210BD0021BA
:10B2100041628169124A01E0B9B1491E01EB810323
:10B2200052F82330002BF7D001EB810302EB8302AD
:10B2300002F1080453685B685360A34201D15B6864
:10B240005360DA680260816110BD502080F311887C
:10B25000BFF34F8FBFF36F8FFEE70000440A00205B
:10B26000A870002070B52020FFF728FD040005D04D
:10B270000025201D2560FFF7DCFD2577204670BDE9
:10B2800038B558B120210446002000912060201DCF
:10B29000FFF7CFFD01202077204638BD502080F3F6
:10B2A0001188BFF34F8FBFF36F8FFEE71CB52649A0
:10B2B00008780190FF20087008788DF800009DF84C
:10B2C00000009DF8002000F0F000904207D05020D0
:10B2D00080F31188BFF34F8FBFF36F8FFEE79DF8A8
:10B2E00000001A4B00F0500018700720986005E02D
:10B2F0009DF8002052008DF80020401E9DF800208F
:10B300001206F5D49860032807D0502080F31188E6
:10B31000BFF34F8FBFF36F8FFEE74FF4407098601D
:10B32000019808700A48016841F4700101600168E1
:10B3300041F070410160FFF711FE00205860F4F702
:10B3400019FF00201CBD000000E400E0B00A00204E
:10B3500020ED00E010B50C4648B184420FD95020D2
:10B3600080F31188BFF34F8FBFF36F8FFEE750203C
:10B3700080F31188BFF34F8FBFF36F8FFEE7022278
:10B38000002100F03CF8002800D0846310BD38B5DF
:10B390000C4648B184420FD9502080F31188BFF386
:10B3A0004F8FBFF36F8FFEE7502080F31188BFF3FC
:10B3B0004F8FBFF36F8FFEE70221134600220091EB
:10B3C000114600F040F8002800D0846338BD10B565
:10B3D00002460021012000F012F80446FFF718FA97
:10B3E000204610BD38B50B460022009011460120C2
:10B3F00000F029F80446FFF70BFA204638BDF8B5EF
:10B4000017460E46050014D0DEB105FB06F050309D
:10B41000FFF754FC04000AD0002084F8460004F131
:10B4200050023B46314628460094FFF7FDF920467E
:10B43000F8BD502080F31188BFF34F8FBFF36F8F9B
:10B44000FEE70020E3E738B5049D18B153B1CAB157
:10B4500081B120E0502080F31188BFF34F8FBFF3FC
:10B460006F8FFEE7502080F31188BFF34F8FBFF33B
:10B470006F8FFEE7502080F31188BFF34F8FBFF32B
:10B480006F8FFEE739B1502080F31188BFF34F8FE3
:10B49000BFF36F8FFEE750241C46012384F846302B
:10B4A0002B460094FFF7C0F9204638BD70B50D4615
:10B4B000040025D0FFF7F0FCD4E90F20216802FB3F
:10B4C000001161600021A1632168A1600A46D4E9EE
:10B4D0000F01401E00FB0121E16021464FF0FF30CB
:10B4E00001F8440F487004F110008DB1FFF7A1FC82
:10B4F00004F12400FFF79DFCFFF7EEFC012070BD76
:10B50000502080F31188BFF34F8FBFF36F8FFEE79A
:10B5100021690029F0D000F00BFB0028ECD0044991
:10B520004FF080500860BFF34F8FBFF36F8FE3E79A
:10B5300004ED00E02DE9FF4782B01D468A464FF03A
:10B540000008040003D0BAF1000F08D011E0502029
:10B5500080F31188BFF34F8FBFF36F8FFEE7206C2E
:10B5600038B1502080F31188BFF34F8FBFF36F8F36
:10B57000FEE7022D0AD1E06B012807D0502080F3AE
:10B580001188BFF34F8FBFF36F8FFEE700F018FAFB
:10B590003F4F4FF000094FF0805648B9049838B13A
:10B5A000502080F31188BFF34F8FBFF36F8FFEE7FA
:10B5B000FFF772FCA06BE16B884207D3022D05D028
:10B5C0000498D0B1B8F1000F1AD01EE02A465146B7
:10B5D0002046FFF774F8616A19B104F1240000F005
:10B5E000A7FA20B13E60BFF34F8FBFF36F8FFFF715
:10B5F00073FC012006B0BDE8F087FFF76DFC22E088
:10B600006846FFF76FFD4FF00108FFF765FCFFF795
:10B61000EFFDFFF741FC94F94400401C01D184F890
:10B62000449094F94500401C01D184F84590FFF7FF
:10B6300053FC04A9684600F027F930B12046FFF713
:10B6400007FB00F0ADFA0020D4E7FFF725FCA06B64
:10B65000E16B884213D1FFF73FFC04F1100004991D
:10B66000FFF74EFD2046FFF7F3FA00F099FA0028A5
:10B670009ED13E60BFF34F8FBFF36F8F98E7FFF708
:10B680002BFC2046FFF7E4FA00F08AFA90E700006E
:10B6900004ED00E02DE9F0471F469046894604007E
:10B6A00003D0B9F1000F08D011E0502080F31188C9
:10B6B000BFF34F8FBFF36F8FFEE7206C38B1502080
:10B6C00080F31188BFF34F8FBFF36F8FFEE7022F18
:10B6D0000AD1E06B012807D0502080F31188BFF316
:10B6E0004F8FBFF36F8FFEE7FFF74AFC5020EFF359
:10B6F000118680F31188BFF34F8FBFF36F8FA06B5C
:10B70000E16B884206D3022F04D0002086F3118813
:10B71000BDE8F08794F945503A4649462046FEF781
:10B72000CEFF681C04D06D1C84F845500120EDE765
:10B73000606A0028FAD004F1240000F0F9F900282A
:10B74000F4D0B8F1000FF1D00121C8F80010EDE7F6
:10B750002DE9F747002683B08A46040003D0BAF1EA
:10B76000000F08D011E0502080F31188BFF34F8FF5
:10B77000BFF36F8FFEE7206C38B1502080F3118843
:10B78000BFF34F8FBFF36F8FFEE700F019F9DFF8BB
:10B79000F4804FF000094FF0805748B9059838B150
:10B7A000502080F31188BFF34F8FBFF36F8FFEE7F8
:10B7B000FFF772FBA56BC5B151462046FEF76CFF43
:10B7C0006D1EA563206950B104F1100000F0B0F9BE
:10B7D00028B1C8F80070BFF34F8FBFF36F8FFFF72A
:10B7E0007BFB012006B0BDE8F087059808B11EB1CB
:10B7F00006E0FFF771FB27E06846FFF773FC0126C0
:10B80000FFF76AFBFFF7F4FCFFF746FB94F94400EF
:10B81000401C01D184F8449094F94500401C01D1AA
:10B8200084F84590FFF758FB05A9684600F02CF80E
:10B83000002820460AD0FFF70BFA00F0B1F92046A5
:10B84000FFF7B8F80028B3D00020CBE7FFF7B2F835
:10B8500090B104F124000599FFF752FC2046FFF750
:10B86000F7F900F09DF90028A2D1C8F80070BFF3E5
:10B870004F8FBFF36F8F9BE72046FFF7E9F900F08A
:10B880008FF995E704ED00E02DE9F0410C46050045
:10B890000FD0B4B1FFF700FB1C4B5A696E681868F3
:10B8A000911B002790F85A0098B1186880F85A70D8
:10B8B0001AE0502080F31188BFF34F8FBFF36F8FD2
:10B8C000FEE7502080F31188BFF34F8FBFF36F8FD7
:10B8D000FEE72068B0F1FF3F08D0D5F800C09B6AB2
:10B8E0009C4509D0964207D8012400E00024FFF7C8
:10B8F000F3FA2046BDE8F081884205D9401A20605D
:10B900002846FFF7EFFBF1E72760EDE7440A002048
:10B910002DE9FF5F8346DDE90E87994616468A4684
:10B920009000FFF7CBF905001CD05C20FFF7C6F9AB
:10B93000040014D00020256384F85900CDE90240AA
:10B94000CDE900874B46324651465846FEF77DFF0B
:10B950002046FEF70DFE012004B0BDE8F09F28460A
:10B96000FFF7CEFA4FF0FF30F6E7F0B585B0DDE92E
:10B970000B640A9DA6B1DCB15C2700972663022602
:10B9800084F85960002604AFCDE90246CDE900579E
:10B99000FEF75BFF2046FEF7EBFD049805B0F0BD17
:10B9A000502080F31188BFF34F8FBFF36F8FFEE7F6
:10B9B000502080F31188BFF34F8FBFF36F8FFEE7E6
:10B9C0000548C16919B1806B18B10020704701208A
:10B9D0007047022070470000440A00200148406977
:10B9E00070470000440A00202DE9F0412E4C00274A
:10B9F000A06B40B1206A401C2062606A00B1012740
:10BA00003846BDE8F0816669761C666113D16068CE
:10BA1000006838B1502080F31188BFF34F8FBFF317
:10BA20006F8FFEE76068A1686160A060A06A401C3B
:10BA3000A062FFF78DF8206BDFF87080864209D393
:10BA40006068006880B16068C068C56868688642E0
:10BA50000DD220632068C06A00EB800158F82100F5
:10BA60000128CAD90127C8E74FF0FF30F1E7281DA8
:10BA7000FFF7B4F9A86A18B105F11800FFF7AEF99D
:10BA8000E86AA169884200D9A06100EB800108EB57
:10BA90008100291DFFF7F3F9E86A2168C96A884225
:10BAA000CED30127CCE70000440A0020A870002074
:10BAB00070B504004FF0000133D01B4D286884425C
:10BAC00007D0502080F31188BFF34F8FBFF36F8FE3
:10BAD000FEE7206D38B1401E2065E36CE26A9A42B1
:10BAE0001FD040B11DE0502080F31188BFF34F8F6D
:10BAF000BFF36F8FFEE7201DFFF770F9E06CE06287
:10BB0000C0F13800A061E06AA969884200D9A86143
:10BB1000064900EB800001EB8000211DFFF7AFF923
:10BB20000121084670BD0000440A0020A8700020D2
:10BB300070B5C068C46854B104F118000646FFF738
:10BB40004DF9144DA86B50B13146134815E0502003
:10BB500080F31188BFF34F8FBFF36F8FFEE7201D77
:10BB6000FFF73CF9E06AA969884200D9A8610B494E
:10BB700000EB800001EB8000211DFFF780F9E06AF7
:10BB80002968C96A884202D90120686270BD002014
:10BB900070BD0000440A002030750020A87000200D
:10BBA0002DE9F0472C4D00242746A86B38B1FFF74C
:10BBB00073F9A86B401EA863A86B40B146E0502003
:10BBC00080F31188BFF34F8FBFF36F8FFEE72969B2
:10BBD000224E0120D1B3A6F5916980463068E0B1CC
:10BBE000F068C46804F11800FFF7F8F8201DFFF7AB
:10BBF000F5F8E06AA969884200D9A86100EB8001E4
:10BC000009EB8100211DFFF73AF9E06A2968C96A4A
:10BC10008842E3D3C5F82480E0E70CB1FEF798FF33
:10BC20002C6A4CB14FEA0806FFF7DEFE00B16E62E7
:10BC3000641EF9D100202862686A38B108490127DA
:10BC400038070860BFF34F8FBFF36F8FFFF744F9DA
:10BC50003846BDE8F0870000440A00203075002017
:10BC600004ED00E02DE9FC4781461E461746884654
:10BC700030200A9DFFF722F804000AD0CDE90054D5
:10BC800033463A4641464846FEF72FFE002084F8E8
:10BC90002C002046BDE8FC877CB53026DDE9065443
:10BCA000009644B1CDE90054FEF71FFE012084F850
:10BCB0002C0020467CBD502080F31188BFF34F8FAD
:10BCC000BFF36F8FFEE7000010B586B0FEF7B8FC3B
:10BCD000114CA068B8B100200390049005AA04A9F3
:10BCE00003A8FFF799F8DDE9032102208DE807009A
:10BCF00000230AA10B48059AFFF737FEE06010B158
:10BD000006B0012010BD502080F31188BFF34F8F83
:10BD1000BFF36F8FFEE70000800A0020546D722091
:10BD2000537663002DAC00082DE9FF411E461346F3
:10BD300002000A9D4FF0000016D0144CA768002F97
:10BD40000FD0CDE900130292062917DAFFF738FE6B
:10BD500002284FF000030FD000226946A068FFF7C9
:10BD6000E9FB04B0BDE8F081502080F31188BFF3F7
:10BD70004F8FBFF36F8FFEE72A46EEE70023324670
:10BD800069463846FFF786FCEBE70000800A002092
:10BD900000C1814001C0804101C0804100C181409B
:10BDA00001C0804100C1814000C1814001C080418B
:10BDB00001C0804100C1814000C1814001C080417B
:10BDC00000C1814001C0804101C0804100C181406B
:10BDD00001C0804100C1814000C1814001C080415B
:10BDE00000C1814001C0804101C0804100C181404B
:10BDF00000C1814001C0804101C0804100C181403B
:10BE000001C0804100C1814000C1814001C080412A
:10BE100001C0804100C1814000C1814001C080411A
:10BE200000C1814001C0804101C0804100C181400A
:10BE300000C1814001C0804101C0804100C18140FA
:10BE400001C0804100C1814000C1814001C08041EA
:10BE500000C1814001C0804101C0804100C18140DA
:10BE600001C0804100C1814000C1814001C08041CA
:10BE700001C0804100C1814000C1814001C08041BA
:10BE800000C1814001C0804101C0804100C18140AA
:10BE900000C0C101C30302C2C60607C705C5C4046A
:10BEA000CC0C0DCD0FCFCE0E0ACACB0BC90908C8DA
:10BEB000D81819D91BDBDA1A1EDEDF1FDD1D1CDCCA
:10BEC00014D4D515D71716D6D21213D311D1D0103A
:10BED000F03031F133F3F23236F6F737F53534F42A
:10BEE0003CFCFD3DFF3F3EFEFA3A3BFB39F9F8389A
:10BEF00028E8E929EB2B2AEAEE2E2FEF2DEDEC2C8A
:10BF0000E42425E527E7E62622E2E323E12120E0F9
:10BF1000A06061A163A3A26266A6A767A56564A4E9
:10BF20006CACAD6DAF6F6EAEAA6A6BAB69A9A86859
:10BF300078B8B979BB7B7ABABE7E7FBF7DBDBC7C49
:10BF4000B47475B577B7B67672B2B373B17170B0B9
:10BF500050909151935352929656579755959454A9
:10BF60009C5C5D9D5F9F9E5E5A9A9B5B9959589819
:10BF7000884849894B8B8A4A4E8E8F4F8D4D4C8C09
:10BF80004484854587474686824243834181804079
:10BF9000ECCD0008000000000000000000000000E0
:10BFA0000000000000020000180000000000000077
:10BFB000000000006CCB0008000000000000000042
:10BFC0000000000000000000000400000800000065
:10BFD0000000000000000000E8CB000800000000A6
:10BFE000000000000000000000000000000400004D
:10BFF00008000000000000000000000058CC00080D
:10C000000000000000000000000000000000000030
:10C010000004000008000000000000000000000014
:10C02000C8CC000800000000000000000000000074
:10C0300000000000000200000800000000000000F6
:10C040000000000014CD0008000000000000000007
:10C0500000000000000000000002000008000000D6
:10C06000000000000000000054CD000800000000A7
:10C0700000000000000000000000000000020000BE
:10C0800008000000000000000000000094CD00083F
:10C0900000000000000000000000000000000000A0
:10C0A0000002000008000000000000000000000086
:10C0B000D4CD0008000000000000000000000000D7
:10C0C0000000000000020000080000000000000066
:10C0D00000000000D8CA00080000000000000000B6
:10C0E0000000000000000000000200000800000046
:10C0F000000000000000000054CB00080000000019
:10C10000000000000000000000000000000200002D
:10C11000080000000000000000000000D0CB000874
:10C12000000000000000000000000000000000000F
:10C1300000020000020000000000000000000000FB
:10C14000F0CA00080000000000000000000000002D
:10C15000000000000000000060CB000800000000AC
:10C1600000000000000000000000000000000000CF
:10C17000DCCB000800000000000000000000000010
:10C1800000000000000000004CCC0008000000008F
:10C19000000000000000000000000000000000009F
:10C1A000BCCC0008000000000000000000000000FF
:10C1B000000000000000000008CD000800000000A2
:10C1C000000000000000000000000000000000006F
:10C1D0001CCB000800000000000000000000000070
:10C1E00098CB0008000000000000000000000000E4
:10C1F00014CC000800000000000000000000000057
:10C2000084CC0008000000000000000000000000D6
:10C21000E4CC000800000000000000000000000066
:10C2200030CD000800000000000000000000000009
:10C2300070CD0008000000000000000000000000B9
:10C24000B0CD000800000000000000000000000069
:10C25000E0CD000800000000000000000000000029
:10C26000E4CA000800000000000000000000000018
:10C2700048CB0008000000000000000000000000A3
:10C28000C4CB000800000000000000000000000017
:10C2900040CC00080000000000000000000000008A
:10C2A000B0CC00080000000000000000000000000A
:10C2B000FCCC0008000000000000000000000000AE
:10C2C00048CD000800000000000000000000000051
:10C2D00088CD000800000000000000000000000001
:10C2E000C8CD0008000000000000000000000000B1
:10C2F00034CB000801000000000000000000000036
:10C30000B0CB0008010000000000000000000000A9
:10C310002CCC00080100000000000000000000001C
:10C320009CCC00080100000000000000000000009C
:10C330000CCB00080000000000000000000000001E
:10C3400088CB000800000000000000000000000092
:10C3500004CC000800000000000000000000000005
:10C3600074CC000800000000000000000000000085
:10C37000D4CC000800000000000000000000000015
:10C3800020CD0008000000000000000000000000B8
:10C3900060CD000800000000000000000000000068
:10C3A000A0CD000800000000000000000000000018
:10C3B000FCCA0008000000000000000000000000AF
:10C3C00078CB000800000000000000000000000022
:10C3D000F4CB000800000000000000000000000096
:10C3E00064CC000800000000000000000000000015
:10C3F00028CB000800000000000000000000000042
:10C40000A4CB0008000000000000000000000000B5
:10C4100020CC000800000000000000000000000028
:10C4200090CC0008000000000000000000000000A8
:10C43000F0CC000800000000000000000000000038
:10C440003CCD0008000000000000000000000000DB
:10C450007CCD00080000000000000000000000008B
:10C46000BCCD00080000000000000000000000003B
:10C4700000000D0510051305160519051C051F05FF
:10C480002205250528052B052E0531053305360522
:10C4900039053C053F054205450548054B054E0558
:10C4A0005105540557055A055D0560056305660588
:10C4B00069056C056F057205750578057B057E05B8
:10C4C0008105840587058A058D05900593059605E8
:10C4D0009A059D05A005A305A605A905AC05AF0510
:10C4E000B205B605B905BC05BF05C205C505C80539
:10C4F000CC05CF05D205D505D805DB05DF05E2055E
:10C50000E505E805EB05EF05F205F505F805FB0582
:10C51000FF050206050608060C060F06120615069C
:10C5200018061C061F062206250629062C062F06BD
:10C530003306360639063C064006430646064A06DA
:10C540004D065006530657065A065E0661066406F7
:10C5500068066B066F067206760679067D0681060A
:10C56000840688068B068F06930696069A069E0614
:10C57000A106A506A906AD06B006B406B806BC0617
:10C58000C006C306C706CB06CF06D306D706DB0612
:10C59000DF06E306E806EC06F006F406F906FD06FB
:10C5A000010706070A070F07140719071D072307C6
:10C5B00028072D07330739073F074507000000000C
:10C5C000000000000000000000000000000000006B
:10C5D000000000000000000000000000000000005B
:10C5E000000000000000000000000000000000004B
:10C5F000000000000000000000000000000000003B
:10C6000000002205250528052B052E0531053405DA
:10C6100037053A053D0540054305460549054C05E6
:10C620004F055205550558055B055E056105640516
:10C6300067056A056D0570057305760579057C0546
:10C640007F058205850588058B058E059205950574
:10C6500098059B059E05A105A405A705AA05AD059E
:10C66000B005B405B705BA05BD05C005C305C605C7
:10C67000CA05CD05D005D305D605D905DD05E005EC
:10C68000E305E605E905ED05F005F305F605FA0510
:10C69000FD050006030606060A060D06100613062B
:10C6A00017061A061D062106240627062A062E0648
:10C6B0003106340638063B063E0642064506480665
:10C6C0004C064F065206560659065C06600663067F
:10C6D00067066A066D067106740678067B067F0695
:10C6E000830686068A068D069106950698069C06A0
:10C6F000A006A406A706AB06AF06B306B706BB06A0
:10C70000BF06C206C606CA06CE06D306D706DB0695
:10C71000DF06E306E706EB06F006F406F906FD067B
:10C72000010706070B070F07140719071D07220744
:10C7300027072B07300736073B07410748074E07F7
:10C74000550700000000000000000000000000008D
:10C7500000000000000000000000000000000000D9
:10C7600000000000000000000000000000000000C9
:10C7700000000000000000000000000000000000B9
:10C7800000000000000000000000000000000000A9
:10C7900000000C050F051205150518051B051E05E3
:10C7A00021052405270529052C052F05320535050A
:10C7B00038053B053E054105440547054A054D053D
:10C7C00050055305560559055C055F05620565056D
:10C7D00068056B056E057105740577057A057D059D
:10C7E00080058305860589058C05900593059605CA
:10C7F00099059C059F05A205A505A805AB05AE05F5
:10C80000B105B405B805BB05BE05C105C405C7051E
:10C81000CA05CD05D005D405D705DA05DD05E00547
:10C82000E305E605EA05ED05F005F305F605FA056D
:10C83000FD050006030606060A060D061006130689
:10C8400017061A061D062006240627062A062E06A7
:10C850003106340637063B063E06410645064806C5
:10C860004B064F065206560659065D0660066406DC
:10C8700067066B066E067206750679067C068006EC
:10C88000840687068B068F06930696069A069E06F2
:10C89000A206A606A906AD06B106B506B906BD06EE
:10C8A000C106C406C806CC06D006D406D806DD06E6
:10C8B000E106E506E906ED06F206F606FB06FF06CA
:10C8C000040708070D07120717071C07210726078B
:10C8D0002B07310736073C074107470700000000D8
:10C8E0000000000000000000000000000000000048
:10C8F0000000000000000000000000000000000038
:10C900000000000000000000000000000000000027
:10C910000000000000000000000000000000000017
:10C92000000018051B051E052105240526052905FF
:10C930002C052F053205350538053B053E0541051B
:10C940004405460549054C054F0552055505580552
:10C950005B055E056105640567056A056D05700583
:10C960007305760579057C057F05820585058805B3
:10C970008B058E059105940597059A059D05A005E3
:10C98000A405A705AA05AD05B005B305B605B9050B
:10C99000BC05BF05C305C605C905CC05CF05D20535
:10C9A000D605D905DC05DF05E205E505E905EC0559
:10C9B000EF05F205F605F905FC05FF050306060679
:10C9C00009060C061006130616061A061D06200692
:10C9D000240627062A062E063106340638063B06AC
:10C9E0003F064206450649064C06500653065706C2
:10C9F0005A065E066106650668066C066F067306D3
:10CA000077067A067E068206850689068D069006DA
:10CA1000940698069C06A006A306A706AB06AF06DA
:10CA2000B306B706BB06BF06C306C706CB06CF06CE
:10CA3000D306D706DC06E006E406E906ED06F206B4
:10CA4000F606FB06FF06040709070D07120717077E
:10CA50001C07210726072B07300736073B0741072E
:10CA60004707000000000000000000000000000078
:10CA700000000000000000000000000000000000B6
:10CA800000000000000000000000000000000000A6
:10CA90000000000000000000000000000000000096
:10CAA0000000000000000000000000000000000086
:10CAB00061636B6E6F776C65676500000000000056
:10CAC000000000000000000001020304060708093E
:10CAD00000000000010203046D795461736B313072
:10CAE000000000006D7954696D65723130000000FE
:10CAF0006D79517565756530310000006D79436F52
:10CB0000756E74696E6753656D3031006D79426979
:10CB10006E61727953656D30310000006D79546932
:10CB20006D657230310000006D794576656E743048
:10CB3000310000006D795265637572736976654DD9
:10CB400075746578303100006D794D757465783095
:10CB5000310000006D795461736B313100000000C9
:10CB60006D79517565756530320000006D795461DD
:10CB7000736B3032000000006D79436F756E74691D
:10CB80006E6753656D3032006D7942696E617279FE
:10CB900053656D30320000006D7954696D657230F7
:10CBA000320000006D794576656E74303200000009
:10CBB0006D795265637572736976654D75746578C4
:10CBC000303200006D794D757465783032000000A8
:10CBD0006D795461736B3132000000006D795175CD
:10CBE00065756530330000006D795461736B3033C7
:10CBF000000000006D79436F756E74696E67536550
:10CC00006D3033006D7942696E61727953656D30B4
:10CC1000330000006D7954696D6572303300000097
:10CC20006D794576656E7430330000006D7952651C
:10CC3000637572736976654D75746578303300007D
:10CC40006D794D7574657830330000006D795175DC
:10CC500065756530340000006D795461736B303454
:10CC6000000000006D79436F756E74696E675365DF
:10CC70006D3034006D7942696E61727953656D3043
:10CC8000340000006D7954696D6572303400000025
:10CC90006D794576656E7430340000006D795265AB
:10CCA000637572736976654D75746578303400000C
:10CCB0006D794D7574657830340000006D7951756B
:10CCC00065756530350000006D795461736B3035E2
:10CCD000000000006D7942696E61727953656D30B4
:10CCE000350000006D7954696D65723035000000C3
:10CCF0006D794576656E7430350000006D794D753F
:10CD000074657830350000006D7951756575653052
:10CD1000360000006D795461736B303600000000FE
:10CD20006D7942696E61727953656D30360000002D
:10CD30006D7954696D657230360000006D79457605
:10CD4000656E7430360000006D794D75746578300D
:10CD5000360000006D795461736B303700000000BD
:10CD60006D7942696E61727953656D3037000000EC
:10CD70006D7954696D657230370000006D794576C4
:10CD8000656E7430370000006D794D7574657830CC
:10CD9000370000006D795461736B3038000000007B
:10CDA0006D7942696E61727953656D3038000000AB
:10CDB0006D7954696D657230380000006D79457683
:10CDC000656E7430380000006D794D75746578308B
:10CDD000380000006D795461736B30390000000039
:10CDE0006D7954696D657230390000006465666163
:10CDF000756C745461736B0018CE0008000000203D
:10CE0000BC0A0000540500086CD00008BC0A0020D1
:10CE100084D20000EC970008A200010004FF0D0A74
:10CE20000001D1011711031810080100003103009F
:10CE300002025300E41010067103003D000C328121
:10CE40001020079BCA51040A0F20135104352008F3
:10CE50001003AE6103000438655B23013918200715
:10CE600055090300D0051700313EAA55AA55010205
:10CE7000030405060708090A0B0C0D0E0F1011120A
:10CE8000131415161718191A1B1C1D1E1F202122FA
:10CE9000232425262728292A2B2CC810098877AA7D
:10CEA0009939019550BC21D20007ED009505AAAA39
:10CEB0000001340421032A0C540AAABBCCDDEEDDA8
:10CEC000CCBB41D409260C52020425F34A0917753C
:10CED000E3080526088A340154231004023006981A
:10CEE000034907580200FF000000401F541F681F3D
:10CEF0007C1F901FA41FB81FCC1FE01FF41F082029
:10CF00001C203020442058206C2080209420A82011
:10CF1000BC20D020E420F8200C21202134214821FD
:10CF20005C21702184219821AC21C021D421E821E9
:10CF3000FC211022242238224C22602274228822D2
:10CF40009C22B022C422D822EC22002314232823BE
:10CF50003C235023642378238C23A023B423C823A9
:10CF6000DC23F023042418242C2440245424682493
:10CF70007C249024A424B824CC24E024F424082580
:10CF80001C253025442558256C2580259425A82569
:10CF9000BC25D025E425F8250C2620263426482655
:10CFA0005C26702684269826AC26C026D426E82641
:10CFB000FC261027242738274C276027742788272A
:10CFC0009C27B027C427D827EC2700281428282816
:10CFD0003C285028642878288C28A028B428C82801
:10CFE000DC28F0280429084F4418292C294029540A
:10CFF0002968297C299029A429B829CC29E029F479
:10D0000029082A1C2A302A442A582A6C2A802A9461
:10D010002AA82ABC2AD02AE42AF82A0C2B202B344E
:10D020002B482B5C2B702B842B982BAC2BC02BD438
:10D030002BE82BFC2B102C2A05FF90053D900D4E64
:10D04000BA0305FF900DFF20030DFF20030D37C22B
:10D0500008EF04080C08063E80FF3F24F4FC060E8F
:0CD060007510C8074FAAAABC0800000009
:0400000508000131BD
:00000001FF
